:10000000C02D0020B9260000B5260000B52600004E
:1000100000000000000000000000000000000000E0
:10002000000000000000000000000000B5260000F5
:100030000000000000000000B5260000B52600000A
:10004000B5260000B5260000B5260000B526000044
:10005000891F0000B5260000B5260000B526000067
:10006000B5260000DD1E0000ED1E0000FD1E000094
:100070000D1F00001D1F00002D1F00001D1500009A
:100080002D1500003D150000B5260000B526000026
:10009000B5260000B5260000B52600008505000045
:1000A000B5260000B5260000B5260000B5260000E4
:1000B0000000000010B5064C2378002B07D1054B3B
:1000C000002B02D0044800E000BF0123237010BDC4
:1000D000B8090020000000001C9B0000084B10B570
:1000E000002B03D00749084800E000BF0748036819
:1000F000002B00D110BD064B002BFBD09847F9E731
:1001000000000000BC0900201C9B00001C9B00009C
:100110000000000010B50022002302704270002190
:100120004280017103760262C26182600373C0245F
:100130006401C481037443748374C37403752A24F3
:10014000035543758375063C0355C2840285C1750A
:100150002B23C1540133C15410BD0000F0B5D64665
:100160004F464646C0B596B0070016000160C64A25
:10017000106A80235B02034313620B780520DB07C0
:1001800005D516B01CBC90469946A246F0BD0B782A
:1001900017309B07F5D473783B71002B04D1BB4A11
:1001A000136C04210B4313640023BB60FB603B61B1
:1001B000BB76FB763B833B77B54B1F602A23F35C12
:1001C000002B05D1337D002B02D101337B7701E079
:1001D00000237B773B68984633786A4613706946FC
:1001E0001E20AC4B98471E20AB4B98472C23F25C4B
:1001F000002A54D0013BF55C337BEB18DBB2D118FD
:10020000C9B28B4221D25219D3B29946A34B9A4616
:1002100003E00135EDB24D4517D00F242C40337B60
:10022000E41850229E4902A8D047132CF1D8A4000C
:1002300002ABE05801A900234B70CB708B700133E7
:100240000B70C0B2974B9847E3E7F489502294496A
:1002500002A8924B9847132C13D9737D9B00DBB2F5
:1002600042461370B37DDB0172781343DBB2424622
:1002700053703379342B00D97BE19B008A4AD358E1
:100280009F46A40002ABE05801A900234B70CB703D
:100290008B7001330B70C0B2824B9847DDE7347B23
:1002A00050227F4902A87D4B9847132C15D9F48919
:1002B00050227B4902A8794B9847132CCDD8A40033
:1002C00002ABE05801A900234B70CB708B70013357
:1002D0000B70C0B2734B9847BFE7A40002ABE05865
:1002E00001A900234B70CB708B7001330B70C0B22F
:1002F0006C4B9847DBE70423102402211AE0717C41
:10030000337C102416E006231024012112E0082378
:10031000102400210EE00023302400210AE00023F5
:100320002024002106E000230024002102E0022313
:1003300010240121090170220A40134342469370A0
:10034000F37D17203F2B00D91BE7D3703A68537E0B
:100350005BB2002BFBDBF37C728813432422B25C7C
:10036000D2001343327D92001343B27C52001343F8
:10037000234342469380337E002B20D0102C00D1A3
:10038000D9E000D898E0202C00D1B6E0302C16D16E
:10039000F27C002A0AD0F26980321720FF2A00D9A5
:1003A000EFE6326A8032FF2A00D9EAE61720F269C6
:1003B000FF2A00DDE5E6326AFF2A00DDE1E6396862
:1003C0004A7E52B2002AFBDB424613723A68537EE1
:1003D0005BB2002BFBDBB38B424693833A68537EC0
:1003E0005BB2002BFBDB338C424613842C23F35C83
:1003F000002B05D0013BDBB217200F2B00D9C0E644
:100400002B22B15C17200F2900D9BAE63868427E4A
:1004100052B2002AFBDBF289307B0243B068024310
:1004200009050A431B041343424613612A23F35C64
:1004300013750F2393751533F35C002B12D0F38CD7
:100440001A4A1720934200D99BE642469384328D84
:1004500080231B01D31815499BB28B4200D990E62B
:100460004346DA84124B1B685B01E022D200134042
:10047000104A516849011268D20E0A43D2B213439E
:100480004246138500207CE600040040000800403E
:10049000980C00205D250000D12400008D40000054
:1004A000589400005526000084930000FF0F0000C0
:1004B0002460800020608000002C00D07FE7F27C68
:1004C000002A0FD0F269802109018C4662442A4932
:1004D00017208A4200D954E6326A624426498A4289
:1004E00000D94EE6244A1720F169914200DD48E622
:1004F000316A914200DD44E661E7F27C002A0FD0C8
:10050000F269802189008C4662441C4917208A4286
:1005100000D936E6326A624418498A4200D930E688
:10052000164A1720F169914200DD2AE6316A9142AC
:1005300000DD26E643E7F27C002A0FD0F269802135
:1005400009028C4662440E4917208A4200D918E6F7
:10055000326A62440A498A4200D912E6084A1720E0
:10056000F169914200DD0CE6316A914200DD08E656
:1005700025E7172005E6C046FF0F0000FF03000037
:10058000FFFF000070B52F4B1D682B681A7EDC7DC5
:100590001440E20716D4630708D504232A681376AB
:1005A000EB7E9B0702D5AB7E9B0742D4A30708D501
:1005B00002232A681376EB7E5B0702D5AB7E5B07CE
:1005C0003BD470BD01221A762A68537E5BB2002BA1
:1005D000FBDB69698B1C6B61538B9BB20B802B8B94
:1005E000013B9BB22B83002B11D06B7F002BD2D011
:1005F0002A68537E5BB2002BFBDB137B02210B438B
:1006000013732A68537E5BB2002BFBDBC3E7012325
:100610002A6893752B7F052BBDD100232B77EB7EAA
:10062000DB07B8D5AB7EDB07B5D52800AB689847AC
:10063000B1E72800EB689847B8E72B69280098478E
:10064000BFE7C046980C0020931C9B001950012363
:1006500093401A00837E13438376704710B5038B53
:100660009BB20524002B01D0200010BD037F052B79
:10067000FAD00523037702834161043B0268D375F6
:10068000437F0024002BEFD00268537E5BB2002B27
:10069000FBDB137B02210B4313730268537E5BB2B7
:1006A000002BFBDB0024DFE7044A137802210B4315
:1006B000137053785BB2002BFBDB704700180040CF
:1006C00000B583B0124A936940210B43936101A99D
:1006D00000230B7005200F4B984705200E4B9847C1
:1006E0000E4A137801210B43137053785BB2002B31
:1006F000FBDB0B4B19004031002204C39942FCD1B3
:100700001022084B1A60084B984703B000BDC04642
:10071000000400405D250000D124000000180040C6
:100720009C0C002000E100E0A9060000002303600B
:10073000436001220272427283720233C3727047B5
:10074000F0B583B005000C0001A900234B70CB70FD
:1007500023790B70237A8B702078154B98470020F3
:100760001F2D00D8134807222A409200E77AA37A67
:10077000002B01D008231F43EB089B00C318996985
:100780000F269640B14397403A000A439A61637A34
:10079000002B06D143690122AA409343436103B071
:1007A000F0BD42690123AB4013434361F7E7C04604
:1007B0005526000000180040F0B5DE4657464E466C
:1007C0004546E0B587B08046049116001F00002220
:1007D000002300218B463F24012021000096019731
:1007E0005C4603944446059413E02024641A0500F3
:1007F000E540A84614E0009C019D121BAB415C46FD
:100800004D462C43A346039C45462C430394013993
:1008100025D3202464420C19E7D40500A540A8463E
:1008200004008C40A14692185B4114001D00059EF7
:100830004F463E40B446049E47463E40B24666465A
:1008400057463E4303D00600264332002B00009C4F
:10085000019D9D42DBD8CED19442D8D8CBE7039BF3
:100860005846190007B03CBC90469946A246AB4694
:10087000F0BD10B5490840230024814202D218007F
:1008800010BD1C00091A631C9BB28842F9D9402391
:10089000FF2CF4D814800023F1E70000F0B583B0FA
:1008A0000F00160008AA117804004C434022BC42F5
:1008B00002D9100003B0F0BD002B14D102000800D3
:1008C0000021194CA04701003A0000230020174CDA
:1008D000A04700220123121A8B41120C1B041A4359
:1008E00032800022E5E70022012BF9D10A00002323
:1008F00000210D4CA04702000B000092019338002C
:1009000000210A4CA047050080239B014022984209
:10091000CFD8790FF800009A019BA047EA00821A0D
:10092000D2B252032A43DBE769290000B90700006D
:1009300010B582B004000E4B1B78002B07D00029A5
:1009400005D10B4B5B78834210D01D200CE001A930
:100950000C701320074B98471320074B9847044B04
:100960005C7001221A70002002B010BD0020FBE76D
:10097000D40900205D250000D1240000404B98429E
:1009800031D00AD93F4B98424DD03F4B98425AD074
:100990003E4B984237D0002070473D4B98420CD0D8
:1009A0003C4B9842F7D1012917D000295DD002298C
:1009B00015D0032915D00020EEE7012907D0002922
:1009C00051D0022905D0032905D00020E4E73248A0
:1009D000E2E73248E0E73248DEE73248DCE7324817
:1009E000DAE73248D8E7012907D000293FD00229A9
:1009F00005D0032905D00020CEE72D48CCE72D48AF
:100A0000CAE72D48C8E7012907D0002931D00229BB
:100A100005D0032905D00020BEE72848BCE72848B8
:100A2000BAE72848B8E7012907D0002923D00229CE
:100A300005D0032905D00020AEE72348ACE72348C2
:100A4000AAE72348A8E7012907D0002915D00229E1
:100A500005D0032905D000209EE71E489CE71E48CC
:100A60009AE71E4898E71E4896E7032094E71D483A
:100A700092E71D4890E71D488EE71D488CE7C04669
:100A80000010004200180042001C00420014004206
:100A900000080042000C00420300050003000600AD
:100AA000030007000300010003001E0003001F00F5
:100AB0000300090003000A0003000B0003001100FB
:100AC000030012000300130003000D0003000E00DA
:100AD00003000F00030017000300180003001900B3
:100AE00003000400030008000300100003000C00D2
:100AF0000300160030B587B00B4B6A4632CB32C2CA
:100B000032CB32C2009B83420BD001239A0069464C
:100B10005258824206D00133062BF7D1002007B08D
:100B200030BD0023D8B2FAE7A894000010B582B017
:100B3000084B98470849094B9847094C0949A04771
:100B40000949A047094B98470190C046019880B2D7
:100B500002B010BDBD29000000247449292D0000F9
:100B6000B92F000000301C4500004842F931000058
:100B7000F0B5ABB01B4E01AC310020001A4B9847CA
:100B80000523E372194B6360022323761848002182
:100B9000184B9847E06101229823E254943BA365E7
:100BA000A3670023A372144D220031002800134BC9
:100BB00098472A68022193681942FCD113680221E0
:100BC0000B4313600A4E002730003900094CA04740
:100BD0000B4B188030003900A0470A4B18802BB00F
:100BE000F0BDC04600200042690F0000C3090000AC
:100BF000DC0500002D0B0000DC0C0020B51000000F
:100C0000DA090020D609002010B582B0364B1B78D7
:100C1000013B012B11D9354B1B88354A1288934271
:100C200003D05CD80133314A1380304B1A8800213D
:100C30003048314B984702B010BD2B4B1B78DBB2CC
:100C4000012B03D0022B28D0002023E02B4B984708
:100C50002B492C4B98472C4B9847A52800DDA52005
:100C60002A4B98472A49274B98472A492A4B9847A5
:100C70002A492B4B9847244B98472A4B181A019026
:100C8000019A294929482A4B98470198C117294BAD
:100C90009847C046164B1880BDE7274B9847184920
:100CA000184B9847184B9847A52800DDA520174BEF
:100CB00098471749134B98471649174B98471F49B0
:100CC000174B9847104B98470400020016491748E5
:100CD000174B9847E1172000164B9847DAE7013B7E
:100CE000024A1380A1E7C046D8090020D609002097
:100CF000DA090020DC0C0020C1140000650E0000A1
:100D00000000C842B92F0000F9310000393200005C
:100D10000080C74300002543292D0000008089443E
:100D2000052A0000270A0000C09400001C0D0020C6
:100D3000D11600002D0B0000910E000000A0BB4456
:100D400010B5064B18701B78002B00D010BD04485E
:100D50000021044B9847044B1880F7E7D80900207E
:100D6000DC0500002D0B0000DA0900200122014BF8
:100D70001A707047DC09002010B500220F4B1A7062
:100D800080320F490F48104B98470C4A1378002BBC
:100D9000FCD00B4B591CFF3100201A8880180233FD
:100DA0008B42FAD1C00980B2084B9847084CE62123
:100DB0008905A0470749A04710BDC046DC090020AF
:100DC000E0090020500D00205D060000D93200002F
:100DD000B92F000068B30E4010B58CB068461A4BAE
:100DE0009847002302936A4653801373C0235B0124
:100DF000D3810023137101235370144C1449200034
:100E0000144B98472268537E5BB2002BFBDB80219A
:100E10000904114B19600F2393751376137802217F
:100E20000B431370094B1A68537E5BB2002BFBDB3C
:100E3000064C002209492000094B9847E37E012215
:100E40001343E3760CB010BD15010000500D0020D7
:100E5000004000425D01000000E100E06D0D000077
:100E60004906000010B5084B1A68537E5BB2002B90
:100E7000FBDB13691F218B431361537E5BB2002B95
:100E8000FBDB024B984710BD500D0020790D000090
:100E900010B5094B1A68537E5BB2002BFBDB13695C
:100EA0001F218B431A390B431361537E5BB2002B16
:100EB000FBDB024B984710BD500D0020790D000060
:100EC000094B98420CD0094B984207D0084A00239E
:100ED000904201D018007047023302E0012300E085
:100EE0000023DBB2F6E7C0460020004200240042A7
:100EF00000280042F8B50F0015001E00046820000D
:100F0000164B9847164B1A5C1723BA4201D81800A3
:100F1000F8BD8000134BC2581723AA42F7D3002E06
:100F200010D080225202BA40236B1A42FCD1802298
:100F30001203BA40A3681A42FCD11C37BF003D51CE
:100F40000023E4E780225200BA40A3681A42FCD191
:100F50001037BF00E41965600023D8E7C10E000018
:100F6000E0940000E894000010B5040008004F4B26
:100F700098470023236080004D4A82586260A37224
:100F8000E372237363722372E36123626362A36279
:100F900023756375A375E375237663762374637491
:100FA000A374E3742C22A3540132A3540132A3543A
:100FB0000132A3540132A3540132A3540132A35489
:100FC0000132A3540132A3540132A3540132A35479
:100FD0000132A3540132A3540132A3540132A35469
:100FE0000132A3540132A3540132A3540132A35459
:100FF0000132A3540132A3540132A3540132A35449
:101000000132A3540132A3540132A3540132A35438
:101010000132A3540132A3540132A3540132A35428
:101020000132A3540132A3540132A3540132A35418
:101030000132A3540132A3540132A3540132A35408
:101040000132A3540132A3540132A3540132A354F8
:101050000132A3544132A354A365A3670132A354C0
:10106000E365E3670132A35423661A3AA3501B32A7
:10107000A3546366173AA3501832A354A366143AD4
:10108000A3501532A354E366113AA3501232A3546D
:1010900023670E3AA3500F32A35463670B3AA35051
:1010A00001210C32A1540132A35410BDC10E000025
:1010B000E8940000F0B5DE4657464E464546E0B59A
:1010C00091B001900C0015000800C34B9847030035
:1010D0000100C248026A9E00C14FF7593A430262BA
:1010E00022681C20920706D511B03CBC9046994658
:1010F000A246AB46F0BD226801271740F4D1B9489B
:10110000325817202E68B242EED36E68B242EBD34B
:10111000E869824200D2B9E1286A824200D2B7E18E
:10112000686A824200D2B5E1A86A824200D2B3E185
:1011300098229446AC4462460892002003E00130B5
:101140000132082808D01678002EF8D0A64E765C1A
:101150008642F4DC1720C7E7002202928020400478
:10116000844602E00132042A0ED0A818007C01282F
:10117000F8D19E48405C904200DA8FE16046904092
:10118000029E06430296EDE79D32AA5C002A04D037
:10119000802212010299114302912A7A511E8A413A
:1011A000920006926A7A012A22D0904AD25C1100FB
:1011B00005923522AA5C8A4200D379E12C21695C30
:1011C0000F2900D974E1287B0A90E87A0B902D2032
:1011D0008246AA44002004970EAE0796C026360128
:1011E000B1468446A046280055460993824635E01C
:1011F000069911430691D8E792024F463A400A43B6
:1012000019798B4603215F4639400A4316435A79C0
:10121000520160210A40324399790902C026B60082
:101220000E401643DA791203E021C9010A40164341
:101230003443039A14432043624607995050042ACA
:101240002AD09A7C0599914200D831E1597A0A3521
:1012500004239B46DC440F2900D929E10906F02329
:101260001B0519402B002E783604FF200004064091
:1012700068788024002800D1049C98780827039778
:10128000002801D104980390D878834610205F4647
:10129000002FB1D10498AFE744465546099B524A06
:1012A000D25C9146514650315046413000270022D1
:1012B0000126B2460226FF36B34680267602B046A5
:1012C000A4461C004B460FE00678002E07D0934240
:1012D00000D8E7E0022E14D056469640374301323C
:1012E00001310230082A10D00E78002EECD0934243
:1012F00000D8D5E04646964037430678002EE9D11F
:10130000EDE75E4696403743E9E799462300644699
:101310006A7E120130211140287E072202401143CB
:101320000022802040020E0002E00132042A0BD08D
:10133000A918097D0029F8D00599914200DCB3E095
:10134000010091400E43F0E7B246019802000432DA
:101350003430002102C28242FCD100220198426353
:1013600082639900224A88500460A022A95C643AF2
:1013700081540DA9AA7A0A701E4AD65C30001E4B11
:10138000984730001D4B98474B46002B3CDD2E0004
:10139000583698339846A84401239946AB464546AB
:1013A000A046089C03E001340436AC422AD02378DE
:1013B000002BF8D00CAB4A469A7000230CAAD370CD
:1013C00013002022B21812781A704A465A703078E8
:1013D00019000B4B9847E6E7C10E000000040040DF
:1013E000D4940000E8940000F4940000E09400001D
:1013F000700D0020E49400005D250000D124000061
:101400005526000044465D460A9B1B030B9A1202B8
:101410001343029A134323600422A3681A42FCD1A7
:10142000FF2323710422A3681A42FCD16B461B7E62
:1014300063710E9BE3600F9B2361A7611D4AA36844
:101440001342FCD15346E3631022A3681A42FCD135
:101450002B686363184AA3681342FCD16B6823644A
:101460000598002822DD1C350021144E32008A40E8
:10147000A3681A42FCD104CD0B0010339B00E31883
:101480005A6001318842F1DC00202DE617202BE65E
:10149000172029E6172027E6172025E6172023E640
:1014A000172021E617201FE617201DE600201BE667
:1014B000172019E640000200800004000001080027
:1014C00010B53C23C35C014CA04710BDF50E0000D5
:1014D000F0B5C64600B580000E4BC7583B68DE6AC3
:1014E000BB6B7A6B13401E4000240B4B984602E006
:1014F0000434302C0AD04346E5583542F8D03B1925
:101500005B68380098473B68DD62F1E704BC9046B1
:10151000F0BDC046700D0020F894000010B500200A
:10152000014B984710BDC046D114000010B50120F2
:10153000014B984710BDC046D114000010B50220E1
:10154000014B984710BDC046D114000010B50749A3
:101550000748084B9847084B1B78002B05D0002202
:10156000054B1A700132054B1A7010BD4C950000E6
:101570001C0D0020D1160000E10A0020E00A002026
:1015800010B507490748084B9847084B1B78022BB2
:1015900005D00222054B1A70013A054B1A7010BD96
:1015A000389500001C0D0020D1160000E10A002033
:1015B000E00A002010B507490748084B9847084B38
:1015C0001B78012B04D00123054A1370054A1370C0
:1015D00010BDC046289500001C0D0020D11600004B
:1015E000E10A0020E00A0020F0B5CE46474680B56B
:1015F00085B08146884617001E000CAB1D7801ACF3
:1016000020000B4B98474B4601934346636027727B
:10161000E67221002800074B9847002229000D9808
:10162000054B984705B00CBC90469946F0BDC046A6
:101630002D070000410700003D1F000010B50021EC
:10164000014B984710BDC046691F000010B582B01D
:10165000124B01930A230093093B002200210A2028
:101660000F4CA0470F4B01930B2300930A3B002222
:1016700000210B20A0470C4B01930C2300930B3B44
:10168000002200210C20A0470A20084CA0470B2074
:10169000A0470C20A04702B010BDC046B515000001
:1016A000E9150000811500004D1500003D160000F1
:1016B000034B1878C0B2002801D000221A7070477E
:1016C000E00A0020014B1878C0B27047E10A002000
:1016D0000EB430B582B004000598124B984783B21F
:1016E000FF2B1AD80204120C01320F4D00212800E2
:1016F0000E4B984706AA0192059928000C4B984773
:101700002800084B984782B229002000094B9847CF
:1017100002B030BC08BC03B01847FA20C000064B2A
:101720009847F5E7A5410000240B00201141000077
:1017300039420000A51B00001D20000070B5284A9A
:101740008023DB05136000235360FF2111810021FA
:101750009372D372012424201454013014540130A4
:101760001354013013549362053013540130135451
:1017700053611382D37611761177517613239376C2
:101780005177184B1363184B536301235B429363E8
:10179000D36380235B03D360E1235B021362134EA8
:1017A00013493000134B984735682800124B98476F
:1017B0001F2318408440114B1C603268D369002BF2
:1017C000FCD12B68022213432B60084C013A0C49D0
:1017D00020000C4B98470C4920000C4B984770BDDB
:1017E000E40A002002001600020017001C0D002071
:1017F0000014004241180000AD1E000000E100E0AE
:1018000011180000B11C00005C950000D11600000A
:1018100070B5064D2A78D2B2054C06492000064B19
:10182000984729002000054B984770BDE20A002028
:101830001C0D002058950000D1160000C91C0000A6
:10184000F0B5DE4657464E464546E0B591B0050038
:101850000C00160029600800BA4B98470200236864
:101860000520DB0706D511B03CBC90469946A24640
:10187000AB46F0BD236817309B07F4D4B249086A21
:10188000971C0123BB4003430B620FA92D27F35D77
:101890000B701432D3B202931800AC4B98470298E5
:1018A000AB4B9847F05D0021AA4B9847F37A6B71D8
:1018B0002423F35CAB712523F35CEB71F37E2B7275
:1018C000337F6B722B68984618009E4B98471430F4
:1018D00000220E2306A98C4663441A80328A0292A3
:1018E0008023DB019A4200D19AE00FD9C023DB01AB
:1018F000029A9A4200D18EE080231B029A4200D0C5
:101900001BE1032306930023079308E080239B0138
:101910009A4200D011E1102306930F3B07933368DE
:101920000593F3689B4673690393337E04932623E0
:10193000F35C9A4673689946002B00D19CE08023A3
:101940005B05994500D180E0737E002B02D0B37E09
:10195000424693730E2306AA944663441B8842466C
:101960009381059B5A461343039A13434A461343F4
:10197000029F1F43049B1B021F4353465B071F43E9
:101980002723F35C002B01D104331F43737E9B029A
:10199000327F52021343727F120213432422B25C3D
:1019A000520413432522B25C12041343B17AF27A33
:1019B000114319433389FF2B00D181E08022520467
:1019C000174319432C23F35C002B03D1624B9B7804
:1019D0009B0701D580231F432A68D369002BFCD1C4
:1019E000434659602A68D369002BFCD143461F60E7
:1019F0000EAB80221A7000225A70DA709A70336B24
:101A00000A93736B0B93B36B0C93F36B02930D936D
:101A100000270AAE63E008230693073B07937EE79F
:101A200033680593F3689B4673690393337E04938D
:101A30002623F35C9A4673689946002B18D08023BE
:101A40005B05994501D0002025E02723F35C002B9E
:101A500000D079E7336A1F00C0B2404B98470100BD
:101A60000E2206AB9C46624438003D4B984712E07C
:101A700008230693002307932723F35C002B0ED043
:101A8000069B0093079B0E2206A98C466244B16A0E
:101A9000306A344FB847002800D0E4E654E7336A90
:101AA0001F00C0B22D4B98470100069B0093079B77
:101AB0000E2206A88446624438002A4FB847EAE757
:101AC000F37E002B00D17DE78023DB041F4379E701
:101AD0002000254B984707E00137042F0DD0F9B2BD
:101AE000BB0098590028F3D0431CF5D00EA908700C
:101AF000000CC0B21D4B9847EEE70023EB602B6152
:101B00006B61AB61EB612B62AB626B620022EB85B8
:101B1000AB853033EA540133EA540133EA540133DC
:101B2000EA542868074B984704001149114B98471D
:101B3000A400114BE550002095E6102306930023E6
:101B40000793ECE6F50A0000000400405D25000064
:101B5000D124000031090000002000417925000057
:101B6000730800009D0800007D0900005526000054
:101B7000D91C0000711E00007C0D0020C2791C23BE
:101B8000002A01D118007047C28D92B2173B002A7B
:101B9000F8D1026811850221137E0B42FCD000238C
:101BA000F0E70000F0B5CE46474680B583B00500AB
:101BB00001911720002A04D103B00CBC904699462D
:101BC000F0BDEB790530002BF6D02C68013A93B2CA
:101BD000994600260127204B984611E0731C9BB2C2
:101BE000019A915D6A79012A17D089B21E002800F6
:101BF0001A4B98474B46013B9BB29946434513D03D
:101C0000237E3B42EAD1144B227E3A42E6D1012B9D
:101C100019D0013B002BF7D1E0E70236B6B2019AAA
:101C2000D35C1B021943E2E7237E9B070DD40A4BCA
:101C30000221227E0A420AD1012B0AD0013B002B4D
:101C4000F7D10020B8E71220B6E70020B4E7002063
:101C5000B2E71220B0E7C046FFFF00007D1B000086
:101C6000F8B504000D00160007680F4B9847A38DC8
:101C70009BB2002B03D00D4B98470520F8BDA685DD
:101C80000A4B9847656205223223E2542E3BBB750E
:101C9000237A002B01D02023BB75637A0020002B10
:101CA000ECD00823BB75E9E749200000892000003B
:101CB000931C9B00C31859603021012393401A00E4
:101CC000435C13434354704710B50122014B9847BE
:101CD00010BDC046611C0000F8B58000624BC558BD
:101CE0002C68E369002BFCD1237EA67D1E403023A7
:101CF000EB5C3122AF5C1F40F30722D5EB8D9BB22A
:101D0000002B1CD0AA6A1378DBB2511CA962697936
:101D100001290ED09BB2DB05DB0D2385EB8D013B4A
:101D20009BB2EB85002B0CD1013323750133A375D6
:101D300007E0517809020B430232AA62EBE7012364
:101D40002375B30706D50223237500223133EA54E5
:101D5000FB071AD4730765D5AB8D9BB2002B5FD000
:101D6000638BDBB21A0714D43F221340002B34D00C
:101D70009A0711D51A223223EA54303B63837B073A
:101D800050D528006B6998474CE02800EB689847CD
:101D9000E0E737221340E9E75A0705D51E22322330
:101DA000EA542E3B6383EAE7DA0705D51322322390
:101DB000EA54313B6383E2E7DA0605D54222322357
:101DC000EA54223B6383DAE720221A42D7D0213239
:101DD0003223EA54123B6383D1E7238DDB05DB0D0D
:101DE000DAB2696A0A706A6A511C69626979012902
:101DF00010D0AB8D013B9BB2AB85002B12D10433CD
:101E0000237500222E33EA54BB070BD528002B691B
:101E1000984707E01B0A53706B6A01336B62E8E76F
:101E200004232375F30604D5102323752376FB06BC
:101E30000ED4B30604D52023237523763B070BD499
:101E4000330704D5082323752376BB0608D4F8BDD1
:101E50002800EB699847ECE72800AB699847EFE763
:101E60002B6A28009847F2E77C0D0020704700009D
:101E7000F0B50A4B1B78002B0CD1094F094E0A4DC7
:101E80000024DE515A1914600433182BF9D10122B1
:101E9000024B1A708000024BC150F0BD240C002090
:101EA000280C00206D1E00007C0D002000B583B0C2
:101EB00009236A4613700133537001339370013361
:101EC000D3700133137101335371034B98476B4641
:101ED000185603B000BDC046F50A000010B5024B0D
:101EE0001B680020984710BD280C002010B5024B3D
:101EF0005B680120984710BD280C002010B5024BEC
:101F00009B680220984710BD280C002010B5024B9A
:101F1000DB680320984710BD280C002010B5024B49
:101F20001B690420984710BD280C002010B5024BF7
:101F30005B690520984710BD280C00201723002A54
:101F400001D0180070478B00064A9B58002B03D025
:101F5000834205D01D23F4E7890088500023F0E771
:101F60000023EEE79C0C00201723002901D0180065
:101F7000704700221F2800D8024A01238340D36003
:101F80000023F4E70018004070B50022104B1A70CF
:101F9000002310491F25104E0D4C0AE00D4908E0A2
:101FA00023780133DBB223700F2B10D800211F2BB5
:101FB000F4D9280018400122824008691042EFD06D
:101FC0000A619B009B59002BEAD09847E8E770BD57
:101FD000940D0020001800409C0C002070B50020DB
:101FE000084B98470500084CFA218900A047074B89
:101FF000186007492800A047064B18600522064BC9
:102000001A6070BD45240000512800000000002027
:1020100040420F000400002010E000E030B5084B03
:102020001C68084A002580214902013807D3002C8A
:10203000FBD05460956013680B42FCD0F5E730BDCF
:102040000000002010E000E00C4B1B68002B06D1C4
:10205000EFF31083002B07D00022094B1A70074AB8
:10206000136801331360704772B6BFF35F8F0022AD
:10207000044B1A700132024B1A70F0E7400C00203A
:10208000440C002008000020084B1A68013A1A602E
:102090001B68002B09D1064B1B78002B05D00122B1
:1020A000044B1A70BFF35F8F62B67047400C00207C
:1020B000440C002008000020F0B583B001AC0125DD
:1020C00065700027A770257021003E20064EB0479E
:1020D0008022D205054B9A612770657021000F2080
:1020E000B04703B0F0BDC046F1200000804400417D
:1020F00000B583B001AB80221A700A785A704A7812
:102100009A708A78DA701900014B984703B000BDC5
:102110005526000010B5082803D880001C4B1B581A
:102120009F46002032E01B4B18692FE01A4B1B6AB8
:102130009B059B0F1948D84028E0164B586925E0AD
:10214000144B1B6800209B0720D513491022CB6835
:102150001A42FCD00F4B1A6824231340042B01D0E1
:102160000F4813E000200F4B98470A4B9B681B0455
:102170001B0C58430AE05023074AD35C00205B073E
:1021800004D5044BD86801E08020000210BDC04691
:102190007C950000480C00200008004000127A00E6
:1021A000006CDC027925000070B50C490B6A0478DC
:1021B000857840780122104080014026B3430343D4
:1021C0002A40D2018020834313430322224012027B
:1021D0000348034013430B6270BDC0460008004033
:1021E000FFFCFFFF082803D88000254B1B589F46A3
:1021F000172044E0234A136A02210B431362002094
:102200003DE0204A936902210B439361002036E0B0
:102210001C4A138A02210B43138200202FE0194A23
:10222000938A02210B439382002028E016490B6811
:10223000022213430B60134B9A8419000E32CB68B1
:102240001A42FCD0104A91680E4BD96252689A62C9
:1022500000229A8419001032CB681A42FCD00A4B33
:102260001B689BB2074A9384002008E0054944227A
:102270008B5C022003438B54002000E00020704759
:10228000A095000000080040480C002030B585B043
:10229000C222D2001A4B9A601A4A53681E218B43FD
:1022A000536001236A4613700024174DE0B269465B
:1022B000A8470134252CF9D103A800244470012536
:1022C00085700470114B98470620114B9847114BAD
:1022D0009847114B1C725C729C72DC7201956B46C4
:1022E0005C7006236A4613701472547269460020AB
:1022F0000A4B984700200A4B984705B030BDC046AE
:1023000000080040004000415D250000A9210000B8
:10231000E5210000252300000004004049230000BF
:1023200001240000064A936908210B4393610122AE
:10233000044B1A7019000B781342FCD17047C04649
:1023400000040040000C004070B5060004000D7849
:102350002D0205434B78002B02D08023DB021D4366
:102360004B7A002B02D080231B031D4348680128B1
:1023700010D9431E184234D1022830D9022300223A
:1023800001325B009842FBD81202324314008023D2
:102390005B031D430B7A002B02D080239B031D435C
:1023A000134A53785BB2002BFBDB124B9847124B5E
:1023B0001E700F4A53785BB2002BFBDB0C4B9C600A
:1023C0001A0053785BB2002BFBDB094A536880216B
:1023D00049020B401D435560084B984770BD0022D1
:1023E000D2E70402344380239B021D43D2E7C04658
:1023F000000C004049200000080C0040892000002B
:1024000010B504000B4A53785BB2002BFBDB0A4B80
:1024100098470A4B1C70074A53785BB2002BFBDBD2
:10242000044A516880235B020B435360044B984776
:1024300010BDC046000C004049200000040C0040C4
:102440008920000070B504001A4A53785BB2002B53
:10245000FBDB194B9847194B1C70164A53785BB23B
:10246000002BFBDB134E7068C004C00E144B984762
:102470000500124B1C707668F602F60F114B1C70AB
:102480000C4A53785BB2002BFBDB0A4B9C6824029E
:10249000240C0D4B9847002E07D1012C07D92100A1
:1024A00028000A4B9847050001E00134E540280068
:1024B00070BDC046000C004049200000040C0040E4
:1024C00015210000080C0040892000005128000060
:1024D00010B50400064B9847064B1C70064A5388FB
:1024E0008021C9010B435380044B984710BDC0465F
:1024F00049200000020C0040000C00408920000030
:1025000010B504000F4B98470F4B1C700F4A5388AF
:102510001B05180F53880E490B40538053880D49F3
:102520000B40538011008022D2014B881342FCD112
:1025300006494A8803020648024013434B80064B73
:10254000984710BD49200000020C0040000C0040DC
:10255000FFF0FFFFFFBFFFFF8920000010B50C78E0
:1025600024020443024B9847A4B2024B5C8010BD86
:1025700001250000000C004010B50400064B9847F0
:10258000064B1C70064B5C882405240F054B9847AE
:102590002000054B984710BD49200000020C004068
:1025A000000C0040892000004524000030B5D3789D
:1025B000002B35D11378802B29D01B068024640290
:1025C000234354780225AC4306D19478002C20D1C3
:1025D0008024A402234341605478013C012C1CD97F
:1025E0000D042D0CA024E4052C431C4384620D0C27
:1025F000D02424062C431C438462D478002C22D19E
:102600005B031CD59378012B1ED0416117E000239A
:10261000D7E7C024E4022343DDE70D4C2340DFE786
:1026200041600C04240CA023DB05234383620C0CC3
:10263000D0231B0623438362D378002B03D1537826
:10264000013B012B02D930BD8161F8E78160FAE7D7
:10265000FFFFFBFF10B50A00C1090023002904D1C8
:102660004309DB0105498C4663441F2420400121B6
:1026700081401800024B984710BDC04600440041FD
:10268000AD2500007047000010B5054B9847054B7D
:102690009847054B9847054B9847054B984710BD01
:1026A0008D220000B920000085260000C106000030
:1026B00085260000FEE70000F8B52A4A2A4B9A4218
:1026C00011D01A00294B9A420DD2294A03339B1A82
:1026D0009B0801339B000022234822498C588450D8
:1026E00004329A42FAD1234A234B9A420AD2D34364
:1026F00021495B1803218B4304339B18002102C23C
:102700009342FCD11D4AFF211D4B8B439360FD3941
:1027100090235B001B4AD1501B4AD3780325AB435F
:1027200002242343D370D3780C27BB4308263343BA
:10273000D370164B987B302290432022104398731D
:10274000997BB943314399739A7BAA4322439A7385
:102750000F4A536880210B4353600E4B98470E4B32
:102760009847FEE71C9B000000000020B8090020ED
:1027700004000020B8090020C00D002000ED00E09A
:10278000000000000070004100500041004800417E
:102790000040004145400000C12700000300064AF8
:1027A0001268002A04D0044A1068C31813607047E6
:1027B0000249014A1160F6E7600C0020C02D00209C
:1027C00070B5174B9847174B98470122164B1A7054
:1027D000BFF35F8F62B6154B9847154B9847154B63
:1027E0009847154B9847154C154D164E07E000209D
:1027F000144B9847144B98470A20144B9847A0470E
:102800000028F7D0A847012807D00028EFD00228D9
:10281000F0D102200B4B9847ECE70120B047E9E7E5
:1028200089260000DD1F0000080000203D17000081
:10283000D90D00004D160000710B0000B11600000C
:10284000C5160000410D0000090C00001D2000000D
:10285000002243088B4274D303098B425FD3030ADF
:102860008B4244D3030B8B4228D3030C8B420DD3F2
:10287000FF22090212BA030C8B4202D31212090280
:1028800065D0030B8B4219D300E0090AC30B8B42BE
:1028900001D3CB03C01A5241830B8B4201D38B036C
:1028A000C01A5241430B8B4201D34B03C01A524111
:1028B000030B8B4201D30B03C01A5241C30A8B4254
:1028C00001D3CB02C01A5241830A8B4201D38B023F
:1028D000C01A5241430A8B4201D34B02C01A5241E3
:1028E000030A8B4201D30B02C01A5241CDD2C30955
:1028F0008B4201D3CB01C01A524183098B4201D3D1
:102900008B01C01A524143098B4201D34B01C01ABB
:10291000524103098B4201D30B01C01A5241C30833
:102920008B4201D3CB00C01A524183088B4201D3A2
:102930008B00C01A524143088B4201D34B00C01A8E
:102940005241411A00D20146524110467047FFE7FA
:1029500001B5002000F006F802BDC0460029F7D0FE
:1029600076E770477047C046F0B5CE464746150437
:102970002D0C2E0080B50704140C3F0C9946030C57
:102980007E435D43674363437F19340CE4199C46DF
:10299000A54203D980235B029846C4444B46514369
:1029A00043433604360C250C24046544A4195918F5
:1029B000491920000CBC90469946F0BD0F4BD0B58C
:1029C0000400994206D9430504D08023C40AE402D6
:1029D0001B011C43080001F055FA0022084B00F0CF
:1029E000D1FF06000F00200001F04CFA32003B003E
:1029F00000F0B8FC01F07EFAD0BDC046FFFF1F001A
:102A00000000F041F0B5C6464E024702760A7B0A46
:102A10004400C50FF7004800984600B5240E2A0070
:102A2000DB00000EC90FBC468D4267D0221A002A77
:102A300000DCA5E000283AD1002F00D193E0511E20
:102A4000002900D0BCE00124DB1B5A0146D59B01C4
:102A50009E09300001F0D8FA05388640844200DD36
:102A60009DE0041B320020200134E240041BA640FC
:102A700033005E1EB341002413435A0704D00F22D3
:102A80001A40042A00D004335A0129D50134FF2CFE
:102A900000D181E02A009B015B0AE4B25B02E405FD
:102AA000580AD2072043104304BC9046F0BDFF2CC7
:102AB000E3D080213800C904084384461B2A00DD86
:102AC00082E020206146D140821A60469040020098
:102AD000501E82410A439B1A5A01B8D45A07CED1DC
:102AE000DE082A00FF2C3AD1002E00D1AEE0802370
:102AF000DB0333435B025B0AFF24CFE7211A002983
:102B000052DD002831D0FF2CB7D080203E00C00419
:102B10000643B4461B2900DDAAE020266046C840D3
:102B2000711A66468E4031004E1EB14101435B185A
:102B30005901D3D50134FF2C00D187E00122784917
:102B40001A405B080B40134397E7002C00D0A7E026
:102B5000002B00D0B6E03B1E62D10026002273029B
:102B60005B0AE4B29AE7140087E7002F4DD0481EB5
:102B7000002857D1634401245A01AFD50224DDE770
:102B8000002A24D1621CD2B2012ADEDDDE1B7201D2
:102B900035D5FE1A0D005CE72A0000237EE73300DE
:102BA000604A241A134068E7002963D1611CC8B247
:102BB00001284EDDFF2949D063445B080C005CE727
:102BC000FF2A41D00A0079E701229B1A84E7002CF2
:102BD0001DD0FF2822D08024E404524223431B2A24
:102BE00000DD8AE01C002025D440AA1A93405A1E1A
:102BF0009341234362460400D31A0D0025E7002EBB
:102C000000D026E700220024A9E70C0035E7002BBE
:102C10004DD0D243002AEDD0FF28E0D16346FF24F7
:102C20000D002AE7FF290FD0010073E7002B61D0C8
:102C3000FF24002F00D120E780224146D203114219
:102C400002D0164200D13B00FF2416E7FF240023E8
:102C500024E7002CEAD1002B58D0002F00D10CE73C
:102C600063445A0100D439E72E4A0C00134004E7AC
:102C700001215CE7002C1ED1002B40D0C943002964
:102C80000BD0FF2836D01B2947DC1C002026CC4067
:102C9000711A8B40591E8B4123436344040047E75C
:102CA000002B18D13B1E2DD00D00FF24E5E63B0084
:102CB00004000D00E1E6FF281CD08024E404494212
:102CC0002343E0E7002F00D1D7E6DE1B72011FD5BA
:102CD000FB1A0D00D1E6FF24002F00D1CDE68022A3
:102CE0004046D2031042AFD01642ADD13B000D009A
:102CF000FF24C2E66346FF24BFE601237AE73B00D8
:102D00000400BAE680260022F603F0E63B00B4E6B3
:102D1000331E00D0E2E6002221E70123BDE7C046D2
:102D2000FFFFFF7DFFFFFFFBF0B557464E46DE4637
:102D30004546E0B544024300C60F83B00F1C640A49
:102D40001B0EB24653D0FF2B27D08022E400D204C2
:102D500014437F22524290469844002399469B4652
:102D60007D027800FB0F6D0A000E009324D0FF282F
:102D700046D080230021ED00DB041D437F38474609
:102D8000381A4F460F43BF00B9463300009A874FA9
:102D900053404A46BA5801939746002C4ED1082317
:102DA0009946F7339846FD3B9B467D027800FB0F22
:102DB0006D0A000E0093DAD1002D26D100200121EA
:102DC0003300009A7A4F53404246101A4A460A434B
:102DD0009200BA581D009746009B2C009A468B46DD
:102DE0005B46022B31D15346FF21002438E0002CF2
:102DF00017D1042399460023984601339B46AFE739
:102E0000FF20002D0BD10221DAE7280001F0FCF8A9
:102E1000431F9D4076235B42181A0021AFE7032130
:102E2000ADE7200001F0F0F8431F9C4076235B42A1
:102E30001B1A9846002399469B4691E70C23994616
:102E4000F3339846FC3B9B468AE7032B00D1A5E071
:102E50005546012B00D081E00123002100242B40A6
:102E60006402C905600ADB070843184303B03CBC91
:102E700090469946A246AB46F0BD80240023E40369
:102E8000FF21EDE7FF210024EAE70123591A1B295E
:102E900066DD019A134000210024E1E78023DB0373
:102EA0001C4238D01D4251D01C436402640A3300D6
:102EB000FF21D5E763016C01A3423BD21B26002111
:102EC000013801251F0049005B00002F01DB9C42F7
:102ED00001D81B1B2943013E002EF3D11C00631EA9
:102EE0009C410C4301007F310029CEDD630704D0F3
:102EF0000F232340042B00D00434230103D5010009
:102F00002C4B80311C40FE290DDD0123019AFF214D
:102F100013400024A4E78023DB031C436402640AFB
:102F20003300FF219CE70123019AA401640AC9B27E
:102F3000134095E71B1B1A260121C2E7009B8B4615
:102F40009A4600244CE76302E5D500258024E4037B
:102F50002C436402640A009BFF2181E70195C1E7CD
:102F600023002020CB40411A8C40611E8C411C4321
:102F7000630704D00F232340042B00D004346301E3
:102F800005D50123019A01211340002468E701239C
:102F9000019AA401640A1340002161E78023DB0346
:102FA0001C436402640A5346FF2159E7C49500009C
:102FB00004960000FFFFFFF7F8B557464E4645461A
:102FC000DE46E0B54702460088467F0A360EC40F4B
:102FD000002E47D0FF2E24D0FB008027FF041F4384
:102FE000002399469A467F3E43465D025800DB0F18
:102FF0006D0A000E984643D0FF283BD0EB00802599
:103000000022ED041D437F383618731C41469B4651
:103010004B46614013430F2B64D875489B00C3583F
:103020009F46002F42D108239946063BFF269A4629
:10303000DAE74146022A28D0032A00D1CEE0012A4D
:1030400000D0ACE0114000200022CCB24002D205FA
:10305000400AE407104320433CBC90469946A246F0
:10306000AB46F8BD002F15D104239946033B00263B
:103070009A46B9E7FF200222002DC5D00322C3E7FC
:10308000002D19D100200122BEE70124FF220C40AF
:103090000020DBE7380000F0B7FF7626431F9F4093
:1030A00000237642361A99469A469DE70C239946A4
:1030B000093BFF269A4697E7280000F0A5FF431F2B
:1030C0009D4076235B42181A00229DE78020002451
:1030D000C003FF22BAE73D005246ABE73D002100A6
:1030E0005246A7E73B0C9C462A04120C2B0C1400FA
:1030F000604665463F043F0C7C4342435D437B434F
:10310000270C9B18FF18BA4203D980235B029C4608
:10311000654424043A04240C121993015C1EA34153
:103120003F0C920E7D191A43AD0115432B0104D5B6
:1031300001235E466A081D40154332007F32002A93
:1031400025DD6B0704D00F232B40042B00D0043562
:103150002B0103D53200274B80321D40FE2A94DC20
:103160000124A801400AD2B20C406FE78020C003BE
:10317000074207D0054205D128434002400A444691
:10318000FF2263E738434002400AFF225EE7012442
:10319000A31A1B2B05DD0C400022002056E75E46DB
:1031A000CBE72A002020DA40C31A9D402B005D1E89
:1031B000AB4113435A0704D00F221A40042A00D00F
:1031C00004335A0104D5012401220C4000203DE7BC
:1031D00001249B01580A0C40002237E7802001247B
:1031E000C00328434002400A0C40FF222EE7C0469D
:1031F00044960000FFFFFFF741024300C20F490A57
:103200001B0E00207E2B0DDD9D2B0CDC802000048E
:103210000143952B0ADC9620C31AD9404842002A64
:1032200000D108007047034BD018FBE7963B99404C
:10323000F4E7C046FFFFFF7F70B5002830D0C3170A
:10324000C4185C40C50F200000F0DEFE9E231B1A50
:10325000962B0DDC9622D21A94402A006402640A4E
:10326000DBB26402DB05600AD2071843104370BD6D
:10327000992B19DC9922D21A002A29DD94402200C8
:10328000144C1440510704D00F210A40042A00D0E6
:103290000434620113D4A401640ADBB22A00E0E71B
:1032A000002200230024DCE705222100121AD1406D
:1032B000B922D21A9440621E94410C43DAE7054BBE
:1032C0002A001C409F23A4011B1A640ADBB2C8E732
:1032D0002200D5E7FFFFFFFB10B5041E27D000F04A
:1032E00093FE9E231B1A962B0ADC9622D21A944038
:1032F0006402640ADBB26402DB05600A184310BD95
:10330000992B17DC9922D21A002A27DD944022003B
:10331000134C1440510704D00F210A40042A00D056
:103320000434620112D4A401640ADBB2E3E700238F
:103330000024E0E7B9222100D21A91400A00511E70
:103340008A410521091ACC401443DBE7044B1C4099
:103350009F23A4011B1A640ADBB2CCE72200D7E743
:10336000FFFFFFFBF8B54546DE4657464E460C03C9
:10337000E0B54E00C90F88460D00610A440F0C43AA
:10338000C70019035800DB0F9B464B0A510F0B4334
:10339000760D400D1900D200D84500D1AEE0351AA7
:1033A000002D00DCF6E000280FD1134300D1DBE054
:1033B0006B1E002B00D037E1BA1A9742BF41641A46
:1033C0007F42E41B0126170024E0C64B9E424DD0ED
:1033D00080231B041943382D00DD07E11F2D00DD7C
:1033E00038E12020431B9A460B0050468340994603
:1033F00013004846EB401843030050468240501EDD
:103400008241E9401A43BA1A611A9742A44117004F
:1034100064420C1B230262D56402650A002D00D1B0
:10342000DFE0280000F0F0FD0300083B1F2B00DD6B
:10343000D2E020223C00D21A9D40D4409F40254338
:103440009E4200DDC4E09E1B731C1F2B00DDF1E0DB
:10345000202238002900D21AD840914097402C00F1
:103460000143781E8741DC4000260F437B0709D0CB
:103470000F233B40042B05D03B1DBB42BF417F4285
:10348000E4191F0023022CD5964B01369E4200D131
:103490009AE04546944BFF081C406007760564029D
:1034A0000743240B760D00212403230B0C0D8F4AB8
:1034B00024051C431440330523435B00ED075B08E0
:1034C0002B43380019003CBC90469946A246AB46B7
:1034D000F8BD6446044300D111E2040067467B074F
:1034E000C6D145466007FF080743E4087D4B9E426E
:1034F00030D024037605240B760DD4E7331A9A4690
:10350000002B78DD002831D076488642AED080206E
:10351000000401435346382B00DCE9E00A43511E06
:103520008A410021D219BA42BF4109197C421700D1
:103530000C192302D3D56B4B01369E4200D13AE1E0
:103540000120694B1C407B0807401F43E0070743ED
:1035500064088BE723003B4300D1CBE180221203B8
:1035600014432403240B9EE72E007FE7080010433A
:1035700000D1B4E0581E002800D0DEE0BA18BA42EC
:103580009B4164185B42E418170001262302A6D56C
:103590000226D5E7002D6ED1701C4005400D012894
:1035A00000DCF9E0B81A844687428041E51A4042BF
:1035B0002D1A280200D489E0D71BBA4292411C1B65
:1035C0005242A51AD84629E74546002400276AE753
:1035D000454CF61A2C4049E73D0028388540002725
:1035E0002EE7380000F010FD20301DE70A43511E81
:1035F0008A41002107E7002B00D0F3E0701C43054F
:103600005B0D012B00DCADE0364B984200D1D1E0E0
:10361000BA18BA42BF4164187F42E419E70752085A
:1036200017436408060021E72E48854200D193E045
:103630001D00D0E629001F3EF140202B00D18DE077
:103640004022D31A9D402F437D1EAF4100240F43DB
:10365000002644E72B000800203BD8400300202D23
:1036600000D17DE04020451BA9400A43511E8A41FC
:1036700000211A43C7E6002E50D01A4EB04257D050
:1036800080266B429946360434434B46382B00DD86
:10369000D6E01F2B00DD35E12026F51A2600AE40CE
:1036A000B2463E00DE40AC46350056462E436546E7
:1036B000AF407D1EAF41DC403743D71BBA42924139
:1036C0000C1B5242A41A0600D846A3E6644667467D
:1036D0002C4300D0A2E600250026002706E71E00A6
:1036E000C4E6C046FF070000FFFF7FFFFFFF0F801B
:1036F0001F2B63DC2020C31A080098409C46834699
:1037000053461000D84003005846184363469A4079
:10371000531E9A4153460243D94003E726003E43D5
:1037200006D0EB439946002BC7D0944EB042ACD1A3
:103730000C0017000600D84698E6904B9A450BD02F
:103740008246E7E6002800D09EE01800104300D132
:10375000E9E01C001700D846884E87E6002572E78E
:10376000002182E723003B43002E00D0ABE0002B7A
:1037700000D1E7E00B00134300D177E6BA18BA4254
:10378000BF4164187F42E419230200D4F2E07C4B6D
:1037900017001C40060069E620003843002ED1D1F6
:1037A00000285BD11C00144300D1A8E01C001700C6
:1037B000D8465BE606000024002797E650460B003B
:1037C0002038C34099465346202B00D195E0402332
:1037D00050461B1A99400A43511E8A414B4600210C
:1037E0001A439FE6002E30D126003E4367D0DB43CC
:1037F0009A46002B1CD0614EB04260D05346382B05
:1038000000DD96E01F2B00DD9FE02026F31A260046
:103810009E409C46B34653463E00DE4033005E4623
:103820001E4363469F407B1E9F415346DC40374307
:10383000BF189742924164185242A418060078E6D5
:1038400027437C1EA741002437E74C4EB04236D0B8
:1038500080265B4236049A463443CFE71800104373
:1038600000D103E6B81A84466745AD41E01A6D42BF
:10387000401B050200D42CE6D71BBA4292411C1B08
:103880005242A41AD846F1E51800104300D163E76C
:10389000F808670707438020E4080003044208D0C3
:1038A000DD08054205D1D208590711430F002C004D
:1038B000D8467B0FE4001C43FF00304ED6E50C00D9
:1038C00017000600D2E5002B38D00B00134300D1BF
:1038D00042E7F808670707438020E4080003044232
:1038E000E7D0CB080342E4D1D208490711430F00C7
:1038F0001C00DEE700270024D5E500216BE700254A
:103900000027F3E54E462500203EF5404B462E00AD
:10391000202B2DD04025ED1AAC4027437C1EA7411B
:1039200000243743C9E6802400252403134E0027D2
:10393000DCE527437C1EA741002479E70C00170033
:103940000E4E93E50C00170090E556462300203EEE
:10395000F34099465346202B0ED0402356469B1BDE
:103960009C4027437C1EA7414B4600241F435FE732
:103970000024D2E71700B2E50024F2E7FF070000B9
:10398000FFFF7FFFF0B557464546DE464E46E0B5A1
:103990000C0398464E00230B87B0070092469B46C7
:1039A000760DCD0F002E6BD06D4B9E4235D080240E
:1039B0005B46420F2404DB0014431C43C3009946BA
:1039C000684BA3469C460023002766440293434667
:1039D0001C035A00DB0F5046240B520D984600D1B1
:1039E00076E05F4B9A426DD08023410F1B040B435E
:1039F0005C49E4008C461C43C300002062444146FD
:103A0000B6186940721C0191944607430F2F00D9E4
:103A1000B0E0554ABF00D25997465B4603439946EA
:103A200000D087E000239B46023308270293CEE7AD
:103A300042460192022867D0032800D10EE20128F5
:103A400000D062E100230024002299460199014040
:103A5000CDB2002112030B0D120B1B051343434A79
:103A6000240513401C436400ED0764082C434846BA
:103A7000210007B03CBC90469946A246AB46F0BD3B
:103A8000034399464FD05B46002B00D189E158464D
:103A900000F0BAFA03000B3B1C2B00DD7AE11D227B
:103AA000D31A3A0001005C46DA4008398C40130012
:103AB0008F4023439B46B94600232D4E0027361ADC
:103AC000029384E7534623432AD10024022096E739
:103AD0005346234320D0002C00D157E1200000F0B2
:103AE00093FA03000B3B1C2B00DD49E11D21CB1A8F
:103AF00051460200D9405346083A944093400C4343
:103B00001B4A121A00207AE70125019B144C1D4024
:103B10000023002299469CE70024002201206EE742
:103B2000534603206BE700239B46013304270026FE
:103B300002934CE7032381460C27029347E7802238
:103B40000023002512039946054C82E75C464B464C
:103B500002986FE75C464B46019502986AE7C046BB
:103B6000FF07000001FCFFFF84960000FFFF0F80AD
:103B70000DFCFFFF4A464946170C1A0C1B041B0C90
:103B800008041900000C41431500884619007D43C4
:103B90007943039589462900150045434D44029514
:103BA00045462D0CAA46029D5544A94506D98A468C
:103BB000802149028946CA4451460391290C049147
:103BC000414609042D04090C88462900250C2404CB
:103BD0004144240C0591210041438846210079434A
:103BE0008A466843414650448146080C48446F4326
:103BF000824503D98021490289464F44010C8946F8
:103C000039004944029141460F0404993F0C88460B
:103C10000004C01980444146049159460F0C090420
:103C2000090C884659438A46390051438946414622
:103C30004A435146090C8B467B43D2185A4493425F
:103C400003D980235B029B46D94451460904090CE1
:103C50008A46414661437C43130C12044B44524450
:103C6000A1468A463C0041466C434D4351464D4473
:103C70000F0C7D19A94503D9802149028846444487
:103C8000049F0399B84641448B4683458041414295
:103C90008846514608042F04000C3F1858460299E4
:103CA00010188946904292414F44BA465242994672
:103CB0009346C244D144CB448F42BF41C24589415F
:103CC00099459B41934592417F4249422D0C524276
:103CD0000F435B4213437F19FF185B463C19DB0D12
:103CE000059A64021C43430213435D1EAB415A46CE
:103CF000C00D034352021343E20156D501205A0876
:103D000003401343E207134364085A486044002801
:103D10004DDD5A0709D00F221A40042A05D01A1D7A
:103D20009A429B415B42E4181300E20104D58020D3
:103D3000514AC00014406044504A904200DDE3E61E
:103D40000125DB0862071A436402019B9146220B9E
:103D50004405640D1D407CE6802259461203114241
:103D600008D0144206D122431203120B454699464D
:103D7000434C6EE65B461A431203120B404C68E656
:103D800003005446283B9C400023B9E600F03CF970
:103D90002030A6E60300283B9F400023BB469946FF
:103DA0008AE600F031F9203074E6B446ADE701252B
:103DB0002A1A382A06DD019B00241D400023002218
:103DC000994646E61F2A21DC20252000AD1A1E0058
:103DD000AB40A840D6405D1EAB4130431843D440B1
:103DE000430709D00F230340042B05D00300181DFF
:103DF00098429B415B42E418230221D50125019B97
:103E000001241D4000230022994622E61F2521009F
:103E10006D42281AC1400800202A1DD05F35AA1A19
:103E2000944023435C1EA341072503431D40002209
:103E3000002D09D00F2200241A401800042AD6D1E0
:103E4000030065076402220BDB082B43012599461A
:103E5000019B00241D40FCE50024E2E780220125AF
:103E60001203224301991203120B0D409946044C90
:103E7000EFE5C046FF030000FFFFFFFEFE07000066
:103E8000FF07000010B5041E28D000F0BDF8154B48
:103E9000154A1B1AD21A1F2A15DD144AD21A944049
:103EA000002224035B05240B5B0D0021100024037A
:103EB0000A0D240B120522430D4C1B05224013430F
:103EC0005B00590810BD210091400A000B21081A1F
:103ED000C4405B052403240B5B0DE6E700230024AC
:103EE0000022E2E71E040000330400001304000077
:103EF000FFFF0F80F0B54C00640D0B03621C450FF3
:103F00005B0A52052B43C90FC500520D012A28DD5B
:103F10003A4AA618FE2E1BDC002E3EDD8001020070
:103F2000501E82416D0F2A43DB0013435A0704D011
:103F30000F221A40042A00D004338022D2041A40EF
:103F40005AD00136FF2E03D09B015B0AF4B201E088
:103F5000FF2400235802E405400AC9072043084310
:103F6000F0BD002C07D01D43F2D08020DB00800480
:103F70000343FF26DAE72B4303D00523DB08FF2C9E
:103F800003D05B025B0AE4B2E4E7002B32D080206E
:103F9000C00303435B025B0ADCE73200173214DB29
:103FA00080221E2712041343BF1B1F2F0FDC144A4D
:103FB000944664442A00A5402E00A340751EAE41DD
:103FC000FA40334313430026B0E70024D5E702222A
:103FD0005242961B1A00F240202F09D0094884460D
:103FE0006444A3402B435D1EAB41002613439DE771
:103FF0000023F7E70023ADE73400BFE780FCFFFFB5
:1040000082FCFFFFA2FCFFFF1C2101231B0498423E
:1040100001D3000C10391B0A984201D3000A083959
:104020001B09984201D30009043902A2105C401810
:104030007047C046040302020101010100000000B4
:104040000000000070B50D4E0D4D0024AD1BAD10ED
:1040500005D0A300F35801349847A542F9D105F0E3
:1040600047FD084E084D0024AD1BAD1005D0A30040
:10407000F35801349847A542F9D170BDFC9A00006D
:10408000FC9A0000FC9A0000049B0000F0B50500BB
:104090000F2A2FD90B0003439B0734D116000C00C5
:1040A0000300103E350901352D01451927681F60B1
:1040B00067685F60A7689F60E7681034DF6010334F
:1040C0009D42F3D10F239E43103685198919134061
:1040D000032B1AD91E1F0023B4080134A400CF58A3
:1040E000EF500433A342FAD10324A643331D2240E8
:1040F000C918ED18002A05D00023CC5CEC5401331C
:104100009342FAD1F0BD0500F6E71A00F2E7C04687
:10411000F0B5830743D0541E002A3FD0CEB2020030
:10412000032502E01A00013C38D3531C16702B42C1
:10413000F8D1032C2AD9FF220A40150215432A047C
:1041400015430F2C14D927001A00103F3E090136E1
:1041500036019E19156055609560D5601032964203
:10416000F8D10F2297431037DB191440032C0DD9D7
:104170001A00271FBE080136B6009E1920C2B2429F
:10418000FCD1032297430437DB191440002C05D0DF
:10419000C9B21C19197001339C42FBD1F0BD140047
:1041A0000300C6E710B5830725D00378002B24D081
:1041B0000300032102E01A78002A1AD001330B42CF
:1041C000F9D119680E4A0F4C8A188A43224206D147
:1041D000043319680A4A8A188A432242F8D01A001E
:1041E0001B78002B03D0013211780029FBD1101A63
:1041F00010BD181AFCE70300E3E70020F8E7C0460B
:10420000FFFEFEFE8080808030B59BB0009104915F
:1042100008496D4602910591012182244942E981B4
:10422000A4006946AC8100F045F80023009A1370A1
:104230001BB030BDFFFFFF7F10B504001300034A21
:1042400010680A002100FFF7DFFF10BD0C000020FE
:10425000034B10B5002B02D0024800F005F810BD4A
:10426000000000007942000010B501000023002288
:10427000002001F023FB10BD70B5094B094CE41A76
:10428000A41009D0084AA518AD00ED182B68013C10
:104290009847043D002CF9D105F034FC70BDC046B0
:1042A000109B0000149B0000FFFFFF3F7047C046BB
:1042B0007047C046F0B5DE46454657464E46E0B527
:1042C000C3B00D00069114000F93099002F0DEFBBD
:1042D000036818001993FFF765FF1890AB891B0658
:1042E00005D52B690793002B01D101F063F832ABA0
:1042F00025930023A34625AFBB607B6014931693E0
:10430000159332AE17931A930A935B461B785C465B
:10431000002B1CD0252B02D119E0252B03D0013412
:104320002378002BF9D15B46E51A10D05B46336049
:10433000BB6875605B19BB607B6801337B60072BD2
:104340002EDC08360A9B9C46AC4463460A932378CD
:10435000002B2ED0631C9B46002316AAD377012284
:1043600052429246002200210B9220329146203286
:1043700063788846002000249446594601311A008B
:10438000203A582A00D9FDE2D74D9200AA58974604
:104390000B9B0F925B420B9304231C430B78EDE7BE
:1043A0003A000699099803F0DDF9002809D132AEE8
:1043B000C8E7BB68002B04D03A000699099803F0BF
:1043C000D1F9069B9B895B0601D501F0CEF80A98CE
:1043D00043B03CBC90469946A246AB46F0BD012294
:1043E0000B7890462B20C9E74B1C9B460B782A2B59
:1043F00001D101F01BFA1A000021303A8A465946D1
:10440000092ABCD80300110050465A469A46A346D2
:1044100083001B1814785B0058182100531C303996
:104420001A000929F4D952461900824623001000C7
:104430005C46A4E780231C430B789FE78B464146EC
:104440001293002901D001F01FFA10231C430F9A88
:10445000A30601D500F088FEE30601D500F080FD3B
:10446000630601D400F07CFD0021535E0C930432FE
:10447000DB170D930F9201D500F086FE0C990D9A73
:10448000080016ABDB7F104398460200012351461B
:10449000013100D1FFE08021200088430890002AEC
:1044A00000D0FCE05246002A01D000F02CFC002B8A
:1044B00001D000F004FD012032AB20400E9011939A
:1044C00008D02723302128AAD15416AA944648336D
:1044D0006344119353460E9A0793924500DA07926C
:1044E000002313934346002B02D0079B013307930D
:1044F0000223089A1A40914602D0079B0233079381
:104500008423089A1A40109200D04DE20B9B079A20
:104510009C1A002C00DC47E27449BA687B68884624
:10452000102C1FDD31001025464603E0103C0831F9
:10453000102C15DD103201330E604D60BA607B60C7
:10454000072BF3DD3A000699099803F00BF90028D0
:1045500000D036E7103CBA687B6832A9102CE9DC41
:10456000B0460E00414674600133A4183160BC604F
:104570007B60072B01DD00F0A8FC16ABDB7F083663
:10458000984612E28B4641461293002901D001F071
:1045900077F907220F9B07339343013294469C44DB
:1045A00062460F921A6816925B6801221593159B5A
:1045B000169D5B005B08984652424D4B28004146D1
:1045C00004F03EFE002801D000F0FDFD0122484B22
:1045D00052422800414603F0EBFD002801D000F0D4
:1045E000F2FD002200231698159903F0D7FD00284C
:1045F00001D001F022F816ABDB7F9846129B472BC7
:1046000001DD00F0C7FE3B4B119380239C437D3BB3
:1046100007930E93002308949A46139362E70022AF
:10462000303B15001A000300079408002C009B463D
:10463000A3001C190378640014191A000131303AE0
:104640000800092AF4D90B945846079C97E60823DA
:104650001C430B7892E6129310231C438B46A3064F
:1046600000D57BE1E30601D500F07EFC630601D4B2
:1046700000F07AFC0F9B1A880C92002204330F93EF
:1046800000230D920C9A002116A8C1778846514646
:10469000013100D0FFE6002A00D135E30894012B58
:1046A00000D1E5E3022B00D062E3179C0F20A14666
:1046B000B44632AB19000C9A0D9B04004D461440D1
:1046C0002C5D1E07150901392E430C701C092300AF
:1046D000340032001C43F0D10C920D9332AB5B1AC4
:1046E000119166460E93F5E6C8960000709800009A
:1046F000FFFFEF7F2C980000129310231C438B4682
:10470000A30600D511E1E30601D500F031FC6306F4
:1047100001D400F02DFC0F9B1A880C920022043368
:104720000D920F930C9A0123ADE78B4641461293ED
:10473000002901D001F090F8B84B1793A30600D5DB
:10474000ABE0E30601D500F007FC630601D400F0FE
:1047500003FC0F9B1A880C92002204330D920F93D6
:10476000E30700D4A9E00C990D9A0B0013431A003B
:104770000223002A00D186E730201EA908704825B0
:104780006846401900781C4348707CE78B464146D8
:10479000002901D001F083F8A30601D500F0E9FD5E
:1047A000E30601D500F09BFD630601D400F097FD00
:1047B00069460F9B098D1A680433079211800F9385
:1047C000A3E54B461C430B78D8E512930F9B8B4611
:1047D0001D1D1B6816A91A0011930023CB77002A10
:1047E00001D100F0FBFE5346013301D100F038FE49
:1047F00052460021119802F00BFC002801D100F074
:1048000054FF119BC31A1A000E93DB43DB171A40A7
:1048100016ABDB7F0792984600230F9508949A46C3
:1048200013935FE60F9A1293136828AD07936B46B4
:104830001B7F8B462B70002316A9CB771300043304
:104840000F93002308949846013307930E93002397
:1048500011959A4613934BE68B46414612930029D5
:1048600000D1F4E516ABD877F1E563461C430B782D
:1048700084E50B786C2B01D100F086FD10221443E7
:104880007CE58B4641461293002901D000F0E8FFF9
:10489000634B1793A30600D453E707220F9B0733FC
:1048A0009343013294469C4462460F921A685B68B7
:1048B0000C920D93E30700D555E70C990D9A08006B
:1048C000104302230200DEE68B460F9930220B686C
:1048D0000C9300230D9302331C431EAB1A70483215
:1048E0005A700B0004330F934D4B129217930C9A8E
:1048F0000223C8E601231C430B783FE50F9B1A1DDA
:104900001B680B93002B00DA42E50B780F9235E51C
:104910000B78002800D031E50122203090462DE5AB
:104920008B461293A30600D4EDE607220F9B0733B4
:104930009343013294469C4462460F921A685B6826
:1049400011001A00080010430C910D92012302007F
:1049500099E68B461293A30600D483E607220F9BA9
:1049600007339343013294469C4462460F921A687F
:104970005B6811001A00080010430C910D9200238F
:10498000020080E68B4641461293002901D000F0D8
:104990007FFF129B002B00D10BE528AD2B7000236D
:1049A00016AAD37708944EE7BC684346002B0FD075
:1049B00016AA1F23944663443360012373607B6807
:1049C00001340133BC607B60072B00DDB3E10836A6
:1049D0004B46002B0CD01EAB3360022373607B6808
:1049E00002340133BC607B60072B00DDAFE1083689
:1049F000109B802B00D120E153460E9A9D1A002D6A
:104A00003CDD084A7B689146102D2CDD10222100E8
:104A10009246099C32002E004D4609E03C98000069
:104A20005098000080980000103E0832102E16DDCD
:104A300050461031013315605060B9607B60072B20
:104A4000F2DD3A000699200002F08CFE002800D02A
:104A5000B7E4103EB9687B6832AA102EE8DCA9469C
:104A60000C00350016004A46641901333260756047
:104A7000BC607B60072B00DD51E10836089BDB053D
:104A800000D5B6E0119B33600E9B9C4673607B683B
:104A900064440133BC607B60072B00DD9DE0083679
:104AA000089B5B0741D50B9B079A9D1A002D3CDDA7
:104AB000C44A7B689046102D26DD102221009146C5
:104AC000099C32002E00069D03E0103E0832102E95
:104AD00017DDBC4810311060484601335060B960A2
:104AE0007B60072BF1DD3A002900200002F03AFE3E
:104AF000002800D065E4103EB9687B6832AA102E09
:104B0000E7DC35000C00160042466419013324C668
:104B1000BC607B60072B08DD3A000699099802F01B
:104B200021FE002800D04CE4BC680B9B07998B4207
:104B300000DA0B000A9A94469C4463460A93002CC0
:104B400000D0D6E0002332AE7B60FFF7DEFB149B83
:104B5000012B00DCAEE0119B013433600123736054
:104B60007B68BC6001337B60072B00DDDFE2083629
:104B7000199A01333260189A9846944664447260D8
:104B8000BC607B60072B00DDDEE2083600220023DC
:104B90001698159903F0FCFA002800D0A4E1119DA5
:104BA000149B0135013B35607360E41801239C467A
:104BB000E0444346BC607B60072B00DD8BE0083699
:104BC00021AB33601A9B9C467360434664440133B7
:104BD000BC607B60072B00DC61E73A00069909980E
:104BE00002F0C0FD002801D0FFF7EBFBBC6832AE3D
:104BF00056E7129B652BAADD002200231698159913
:104C000003F0C6FA002800D1E2E06F4B01343360B4
:104C1000012373607B68BC6001337B60072B00DD80
:104C200066E308361F9B149A934200DAA4E1089BBE
:104C3000DB0700D5A0E1BC6832E70B9B079A9D1A01
:104C4000002D00DCD8E6614A7B689146102D25DDF9
:104C5000102221009046099C32004E4603E0103D90
:104C60000832102D17DD40461031013316605060B8
:104C7000B9607B60072BF2DD3A000699200002F054
:104C800071FD002801D0FFF79CFB103DB9687B68DF
:104C900032AA102DE7DCB1460C0016004A46641912
:104CA000013332607560BC607B60072B00DD7EE203
:104CB0000836A1E60123089A134200D04BE773603F
:104CC0007B68119A013301343260BC6098467B6086
:104CD000072B00DC73E73A000699099802F042FDC1
:104CE000002801D0FFF76DFB7B68BC68984632AEA8
:104CF00066E73A000699099802F034FD002800D1D1
:104D000020E7FFF75EFB089C012B00D184E1022B1A
:104D100029D10894002300240C930D94C5E43A0093
:104D20000699099802F01EFD002801D0FFF749FB03
:104D3000BC6832AEA2E63A000699099802F012FD6C
:104D4000002801D0FFF73DFBBC6832AE40E63A00D8
:104D50000699099802F006FD002801D0FFF731FB03
:104D6000BC6832AE44E60894002300240C930D94F2
:104D70000C980D995B4632AA07939146B34600E022
:104D8000A1464A0794464B4665465C1EC608072363
:104D9000CA08354311002A0003403033237028002D
:104DA0000A43EDD10C900D9107995E468B46089908
:104DB0004A461194C90700D53DE132AB1B1B0E9347
:104DC000FFF788FB709800006C9800008098000046
:104DD0001F98002800DC96E2139A1499130090465D
:104DE0008B4200DD88464346002B0CDD119B44447A
:104DF0003360434673607B68BC6001337B60072B84
:104E000000DDB7E308364346DB434246DB17134079
:104E1000139AD31A9846002B00DC28E1102B01DCF2
:104E200000F0E7FCCF4A2100914610227B689246B1
:104E3000099D32004C46464604E00832103E102ED2
:104E400000DC04E150461031013314605060B96059
:104E50007B60072BF1DD3A000699280002F082FC06
:104E6000002801D0FFF7ADFAB9687B6832AAE5E700
:104E70000D9B002B00D1CAE00C9C0D9D32ABB146BE
:104E80001E00200029000A22002303F0AFF9013E92
:104E9000303232700023200029000A2203F0A6F9E4
:104EA000030004000D000B43EBD1320032AB9B1A20
:104EB00011960C940D954E460E93FFF70BFB0023B5
:104EC0000E9332AB1193FFF705FB3A000699099850
:104ED00002F048FC002801D0FFF773FA16ABDB7F25
:104EE000BC68984632AE60E5149B5D1E002D00DC68
:104EF00066E69C4B9946102D29DD102332009A4618
:104F00002E0021004346099C4D4603E0103E083226
:104F1000102E17DD50461031013315605060B96016
:104F20007B60072BF2DD3A000699200002F01AFCA4
:104F3000002801D0FFF745FA103EB9687B6832AA15
:104F4000102EE7DCA9460C003500984616004B46AB
:104F500075603360641929E60F9B1A68FFF7FBFB45
:104F600013680793FFF782FA0F9B1A68FFF784FB19
:104F70000F9B1A68FFF7D1FB199BBA683360189B27
:104F80009C4673607B68624401331400BA607B60A6
:104F9000072B00DD02E20836149B5D1E002D00DCAD
:104FA0007EE5704A7B689146102D25DD1022210098
:104FB0009046099C32002E004D4603E00832103E18
:104FC000102E15DD40461031013315605060B96078
:104FD0007B60072BF2DD3A000699200002F0C2FB4D
:104FE000002801D0FFF7EDF9B9687B6832AAE6E73F
:104FF000A9460C00350016004A4664190133326098
:105000007560BC607B60072B00DC48E5E5E50C9B28
:10501000092B00D930E7089C27220C9B28A93033A4
:105020008B54012316AA94460E936E33634408945E
:105030001193FFF74FFA302B00D10BE23023023AE5
:10504000137032AB9B1A0E931192FFF743FAB046DE
:10505000A14616000C004A463260424644440133E1
:105060007260BC607B60072B00DD9CE208361F9BF2
:10507000149A93424CDB089AD20749D4149A139994
:10508000D31A521A90469A4200DD98464246002AA8
:105090000FDD1399119A8C46624432604246726069
:1050A0007A6844440132BC607A60072A00DD86E2F7
:1050B00008364246D543ED1715405D1B002D00DC38
:1050C000EEE4284A7B689146102D95DD10222100E0
:1050D0009046099C32002E004D4603E00832103EF7
:1050E000102E85DD40461031013315605060B960E7
:1050F0007B60072BF2DD3A000699200002F032FBBC
:10510000002801D0FFF75DF9B9687B6832AAE6E7AD
:10511000199A3260189A944672607A68644401322F
:10512000BC607A60072A00DD30E20836A6E73A0064
:105130000699099802F016FB002801D0FFF741F903
:10514000BC687B6832AE13E53A000699099802F014
:1051500009FB002801D0FFF734F97B68BC6898464A
:1051600032AE13E580980000072307329A430133DB
:105170009C46944463460F93536812680D930C92B7
:10518000002B01DBFFF77AF90C980D9900234242BE
:105190008B4111001A002D2316A8C3770800104375
:1051A0000C910D92984602002C3BFFF770F93A00E3
:1051B0000699099802F0D6FA002801D0FFF701F904
:1051C000BC6832AE18E41699159D0A0008002B0041
:1051D000290004F035F8002800D0E6E253460133F8
:1051E00000D10DE22023129A9A430E92472A00D151
:1051F0001CE180235B0023430893159B002B00DAFE
:1052000021E2169A0793002391461093129B662B76
:1052100000D1FCE1462B00D1DBE00E9A0998453A1B
:1052200013005942594120AB0D0003931FAB029369
:10523000022323AA55441B92049200930195079BD5
:105240004A4600F05FFC129B1190672B00D039E2B8
:10525000119B9846A844E30700D48BE20023002268
:105260004846079902F094FF434600280AD1239B41
:10527000434507D2302140465A1C23921970239B84
:105280009842F9D8119A9B1A14930E9B472B00D180
:10529000F6E0129B652B00DC26E2129B662B00D108
:1052A000F4E11F9B1393149B139A1900914200DDA4
:1052B000D4E1E30700D549E2D343DB1711001A40DC
:1052C000672307920E911293109B002B00D0CFE022
:1052D00016ABDB7F984600239A46FFF703F90F9A37
:1052E0000A9913681960130004330F93FFF70DF840
:1052F0003A000699099802F035FA002801D0FFF724
:1053000060F832AE8EE4DE4B01343360012373600B
:105310007B68BC6001337B60072B7ADC0836002891
:1053200007D1149B002B04D1089BDB0701D4FFF7A6
:10533000B7FB199B3360189B191973607B68B960C0
:1053400001337B60072B00DDF2E1320008320028D8
:1053500000DACCE111980133106014987B60441896
:105360005060BC60072B00DD37E408321600FFF701
:1053700097FB0F990A9A0B681A60D2175A600B00B4
:1053800004330F93FEF7C1FF4B4601311C430B78EA
:10539000FEF7F4FFBB4B1193FFF737F93A0006997C
:1053A000099802F0DFF9002801D0FFF70AF8BC687D
:1053B00032AEF1E54021099801F076FB069B1860BA
:1053C0001861002800D14FE24023069A5361FEF78E
:1053D0008EFF23AB1B93049320AB03931FAB02936D
:1053E0005346019303234A4600930998079B00F014
:1053F00089FB55461190119B9846129BA844462B59
:1054000000D02BE7119B1B78302B16D01F9B9844A4
:1054100024E73A000699099802F0A4F9002801D07F
:10542000FEF7CFFF1F98BC6832AE78E75346002BDB
:1054300000D0DEE601339A46DBE600220023484630
:10544000079902F0A5FE0028E0D101235B1B1F9302
:10545000984403E7119A32AB9B1A0E93FFF73AF880
:105460001198FEF79FFE02000E900300FFF7CDF9A2
:105470002D2316AAD377984600239A46FFF735F8CE
:105480001F9B1393DA1C02DB9A4500DB0BE7129B90
:10549000023B12932C22139B48215D1E16AB9B18D6
:1054A0006A46521812781F951A70002D00DAA4E18E
:1054B0002D212B2316AA52181370092D00DC4CE164
:1054C00016AA3B23944663449A46B146A0465646E4
:1054D00000E0260028000A2102F046FE741E30314A
:1054E000217028000A2102F059FD05000928F0DC8E
:1054F00023004446B0464E46994603003033D8B2A6
:105500004346023B18709A4500D8B4E142461B9BC3
:105510004546991A012307315B4201E0E85C0133FB
:1055200021AAD218D0708B42F8D116A98C462E220F
:105530004B4662449446FB1A634421AA14999B1A71
:105540009C460A0062441A930E92012900DC45E150
:10555000189A0E9B944663441A000E93DB43DB17A4
:105560001A40002307921393AEE601235B420A938D
:10557000FEF72DFF3A000699099802F0F3F800288B
:1055800001D0FEF71EFFBC6832AE3CE43A0006993B
:10559000099802F0E7F8002801D0FEF712FF1F9BE0
:1055A000BC6832AE6AE53A000699099802F0DAF86A
:1055B000002801D0FEF705FFBC6832AE57E53A007F
:1055C0000699099802F0CEF8002801D0FEF7F9FEFE
:1055D000149B1F9ABC689B1A32AE6AE55346079328
:1055E000062B01D906230793079B0F950E930023E3
:1055F00098469A461393244B08941193FEF778FF2C
:105600002023129A9A431A3B0E929A46F1E523AB55
:105610001B93049320AB03931FAB02935346019358
:1056200003234A4600930998079B00F06BFA030096
:105630005344119098465546E4E62D2316AAD37795
:105640009846FEF7DBFF802212069446169B994689
:10565000159B634407932D231093D7E5189A149B49
:105660009446139A63440E93002A00DCCEE01A009D
:10567000DB43DB171A4067230792129324E6C046E8
:105680006C98000030980000649800001F9B1393F2
:10569000002B00DCD5E05246002A00D092E0E20761
:1056A00000D58FE007930E930EE616ABDB7F0F95C8
:1056B0009846534607930E93002308949A461393F3
:1056C000FEF710FF119B9846129BA844472B00D071
:1056D000C4E5E30700D58EE6239B119A9B1A149329
:1056E0000E9B472B00D1CBE61F9B1393D2E644427F
:1056F000103000DBD0E06E481026050003E00832D1
:10570000103C102C38DD1031013315605660B96043
:105710007B60072BF3DD3A000699099802F022F826
:10572000002801D0FEF74DFEB9687B6832AAE7E792
:105730003A000699099802F015F8002801D0FEF702
:1057400040FE1F98B9687B6832AA00E6189A139B3E
:10575000944663441A000E938AE72E21302316AA3A
:10576000521813702B0016AA0131303352181370DF
:1057700022ABE2E6239B85E5A94648460919013399
:1057800010605460B96008327B60072B00DCE1E5F3
:105790003A000699099801F0E5FF002801D0FEF7CC
:1057A00010FEB9687B6832AAD4E5159B002B38DB64
:1057B00016ABDB7F9846129B472B2EDC3D4B11939B
:1057C000FEF723FF189A139B9446634453441A0030
:1057D0000E93DB43DB171A40079275E50123234044
:1057E000139300D0B4E60E9AD343DB171A40079206
:1057F0006AE52F4A7B6891462DE40123139A1B39F1
:105800009D1A16AA2C335218137056E60E9B139A43
:10581000981A431C1A000E932AE7274B1193FEF7A0
:10582000F4FE2D2316AAD3779846C4E70F9B1A1DC2
:105830001B689A46002B36DB4B780F925946FEF7D1
:105840009DFD5346002B01D1E30703D5189B581C3F
:105850000300BBE7012325E716ABD877FEF76CFF03
:1058600016ABD877FFF714F80C23099A13600D3B99
:105870000A93FEF7ACFD16AA2E23944663445CE619
:1058800016ABD877FEF785FE16ABD877FEF7DDFDB1
:1058900016ABD877FFF77DF8054881466DE716AB64
:1058A000D877FEF779FF01235B429A46C4E7C046EA
:1058B000809800003498000038980000F0B54E46FB
:1058C0004546DE465746E0B5364D83B006002868AB
:1058D00098460F009146FEF7E9FC334B1C68A42361
:1058E0005B00E058002852D043681F2B13DC5A1C81
:1058F0000192002E28D1019A02339B0042601F5072
:105900002868FEF7D5FC002003B03CBC90469946C1
:10591000A246AB46F0BD254B002B3DD0C820400031
:1059200000E000BF002837D0A42200235200A15875
:1059300043600160A05040328350043283500133F1
:1059400001930023002ED6D09A00924682444A4604
:10595000882154466250C4225200914681444A46EE
:105960008739994012688B460A4394464A466146F5
:105970001160842241465200A150022EBBD1020088
:105980005C468D32FF3211680C431460B3E720008F
:105990004D30FF30E050A7E72868FEF789FC012072
:1059A0004042B1E738040020C49600000000000027
:1059B000F0B545468046DE4657464E464246E0B57F
:1059C0000C69126985B00B0002910020944200DD41
:1059D00090E014229446634499464A46013CA30051
:1059E000D6181422424493469B4433681500591C30
:1059F0005B4618680192FCF72BFF031E009042D013
:105A0000290000274D460020B146A2463E00040072
:105A10009C462F0008000395634604CF15042D0C07
:105A20005D43120C5A43AD192B0CD21803682D0498
:105A30001904090C0919160C2D0C1204491B120C1F
:105A40001B0C9B1A0A149B1809041C14090C1B0438
:105A5000194302C0B945DFD2039B4E4699465B46C7
:105A60001B685446002B0ED15B46019A043B9A42B8
:105A700004D306E0043B013C9A4202D21968002993
:105A8000F8D043461C610299404601F045FD0028CC
:105A90002FDB4F460020009B019D013300932B68B4
:105AA00002CF1A04120C10180A04120C821A090CE4
:105AB0001B0C5B1A11145B1812041814120C1B0433
:105AC000134308C5BE42EAD20199A3008C46634441
:105AD0001A68002A0DD1043B0A00994204D306E05B
:105AE000043B013C9A4202D219680029F8D043468F
:105AF0001C61009805B03CBC90469946A246AB4656
:105B0000F0BDC046F0B557464E464546DE46E0B5C8
:105B1000016C99B082461D0016001F00002909D0B3
:105B20000123426C93404A608B6001F0E9FA002344
:105B300052461364B846002F37DB0023259A1360C2
:105B40004246D64B1A409A4218D000220023300019
:105B5000390002F01DFB00282FD00123249A136086
:105B6000269B002B00D12AE2CD481860013819B0DD
:105B70003CBC90469946A246AB46F0BDC94B249A20
:105B80001360002E0BD14346180308D1269BC6484C
:105B9000002BECD003000833269A1360E7E7269B1E
:105BA000C248002BE3D0C31CF6E70123259A680006
:105BB0001360430898461F00C2E716AB019317AB6A
:105BC000009332003B00504601F05CFD43468346A3
:105BD0001A0D00D1D6E13B03B54C1B0B1C43B54B52
:105BE00030009846169B21009946002390440F935D
:105BF0000022B14B03F00EF8B04AB14BFDF7C2FEE4
:105C0000B04AB14BFDF7AEFB040040460D0003F077
:105C10006BFBAE4AAE4BFDF7B5FE02000B00200059
:105C20002900FDF79FFB04000D0003F029FB002273
:105C3000039000232000290002F0B0FA002800D0D1
:105C4000B1E20123039C0C93162C10D8A149E30068
:105C5000C9183200086849683B0002F0B3FA00280E
:105C600000D11DE32300013B039300230C934B461B
:105C700042469A1A002306931300013B049300D571
:105C8000A1E2039B002B00DA84E29C460D930023E3
:105C9000049A9946110061440491229B092B00D972
:105CA0008FE10124052B02DD0024043B2293229B7B
:105CB000032B01D100F0CEFC01DC00F092FC229B12
:105CC000042B01D100F040FC01230B93229B052BF8
:105CD00001D000F08BFC239A039B944663440E93FF
:105CE000013307931D1E01DC00F049FD079B984618
:105CF0000023524600215364172D0AD90122043390
:105D00005B0018001430110001328542F8D253466E
:105D10005964504601F0CCF95346186443460A9042
:105D20000E2B00D961E1002C00D15EE11096119795
:105D3000039E002E01DC00F025FD32000F21654B93
:105D40000A40D2009B1836111C685D68F30601D426
:105D500000F0CAFC604B0E401A6A5B6A10981199F9
:105D600002F024FB0323984608900991002E11D0DD
:105D7000594F0123334209D09C463A687B68200082
:105D80002900E044FDF7FEFD04000D007610083701
:105D9000002EEED12200089809992B0002F006FB94
:105DA00006000F000C9B002B09D00022404B300056
:105DB000390002F0F3F9002801D000F0C2FD40469E
:105DC00003F092FA32003B00FDF7DCFD0022434B6A
:105DD000FDF7C8FA424A0B009446634408900991C3
:105DE0000993079B002B01D100F050FC039B1393F8
:105DF000079B12930B9B002B01D100F01DFD129B02
:105E000000205A1E334BD2009B181A685B68354934
:105E100002F0CCFA089A099B02F0FCFE0890099166
:105E20003900300003F02CFA040003F05DFA0200A0
:105E30000B003000390002F0EDFE05000E000A9A5A
:105E40003034511CE7B21491177033000898099947
:105E50002A0002F0B7F9002801D000F0FEFD2A0068
:105E600033000020124902F0D5FE02000B00089812
:105E7000099902F0A7F9002801D000F0E7FD129B74
:105E8000012B01D100F078FC0A9A129B94466344DE
:105E900098464B461293149B994638E00000F07FD9
:105EA0006D9800000F270000909800009C9800005B
:105EB0000000F03F01FCFFFF0000F83F61436F630B
:105EC000A787D23FB3C8608B288AC63FFB799F5013
:105ED0001344D33FC8980000A098000000001C4065
:105EE0000000C0FC0000E03F2A0033000020B94958
:105EF00002F090FE089A099B02F050F9002801D0A8
:105F000000F074FDA146444501D100F033FC08982F
:105F100009990022B04BFDF735FD0022AE4B0890E9
:105F2000099128003100FDF72DFD0D00040003F05C
:105F3000A7F9070003F0D8F902000B0020002900A0
:105F400002F068FE4B463037FFB25C1C1F70089AA7
:105F5000099B05000E0002F021F90028C4D0139B14
:105F600003935946504601F0CBF800232370039B5E
:105F7000249A01331360269B002B00D1A8E31C60F8
:105F80000A98F4E5169B9946179B4B441C00934BCB
:105F9000E318202B00DC7EE13100914A4046A21834
:105FA000D1400A004021CB1A98401043FDF76AFF08
:105FB000631E984601238B4D0F93491918E68A48B2
:105FC000D5E50023524600215364504601F070F895
:105FD0005346186401235B4207930E930233002259
:105FE0000B9300230A9023922293179B002B00DA35
:105FF000ABE0039A0E2A00DDA7E07C4BD2009B1891
:106000005C681B6804930594239B002B00DAA7E2CD
:10601000049C059D300022002B00390002F0C6F9D7
:1060200003F02EF9804603F05FF922002B00FDF704
:10603000A9FC02000B003000390002F0EBFD4346E2
:106040000A9A30331370079B06000F00541C012B73
:106050004ED00022604BFDF795FC00220023060085
:106060000F0002F095F8002800D07AE70A9B079A03
:106070009D1C9C465B46069353466244AA46049C7C
:10608000059D914607930FE00022534BFDF77AFCE4
:1060900001239C460022002306000F00E24402F088
:1060A00077F8002800D0D9E222002B003000390018
:1060B00002F07CF903F0E4F8804603F015F92200C1
:1060C0002B00FDF75FFC02000B003000390002F0EE
:1060D000A1FD53464246013B303206000F00D34635
:1060E0001A70D145D0D1069B54469B46079B9A46D1
:1060F00032003B0030003900FDF734F906000F0094
:1061000002000B000498059902F048F800280CD111
:106110000498059932003B0002F03AF8002800D1BB
:106120001FE74346DB0700D41BE7651E2F780A9B59
:1061300006E09D4200D151E3023C27782C00013D4E
:10614000392FF6D001372F700BE70B9A002A4FD06A
:10615000229A012A00DC2CE2079B5C1E4B46A145DB
:1061600000DAB8E21C1B079B002B00DAD4E3069B85
:106170000893079B069A012194469C446246069226
:10618000049A504694469C446346049301F050F8A8
:10619000804632E0069A039BD21A5B42994600235E
:1061A00006920D9379E5039803F09EF80B00020028
:1061B0002900200001F0ECFF020050425041039BF7
:1061C0001B1A03933DE501239B1A069300230493B6
:1061D00057E5C0460000F03F0000244032040000B4
:1061E00012040000000010FE6C980000C898000027
:1061F000069B4C4608930023984608990B1E0EDD1B
:10620000049A002A0BDD934200DD87E1069AD21A38
:106210000692089AD21A0892049AD31A04934B460B
:10622000002B1AD00B9B002B00D1BBE1002C10DD02
:1062300041462200504601F0AFF85A460100804620
:10624000504600F0FFFF05005946504600F058FF49
:10625000AB464B461A1B00D0A5E10121504600F089
:10626000E7FF0D9B8146002B1DDD1A000100504603
:1062700001F092F8229B8146012B00DC50E10024C2
:106280004B461B6903339B004B44586800F088FF62
:1062900020231B1A10E020223000D31A984085E6F4
:1062A00000230C93E3E4229B0024012B00DC8BE110
:1062B0000D9A0123002AE3D104991F208C466344E0
:1062C000184000D1AEE020231B1A042B00DCCCE3E5
:1062D0001C23181A069B9C46844463460693089B1D
:1062E0009C46844463468C468444089363460493E6
:1062F000069B002B05DD59461A00504601F0ACF80C
:106300008346049B002B05DD49461A00504601F0E8
:10631000A3F881460C9B002B00D094E0079B002B38
:1063200000DC75E10B9B002B00D1A6E0089B002B45
:1063300005DD41461A00504601F08EF8804643467E
:106340000C93002C00D050E2079C0A9A013C2300D9
:106350009446634408930123334007934B460693C6
:106360000C9B574645465E4692469846069B300033
:1063700019009946FFF71CFB03000B9030332900EE
:106380003000049301F0C8F8494604004246380042
:1063900001F0DCF8C3688146002B00D01EE101004B
:1063A000300001F0B9F883464946380000F0A8FEF5
:1063B0005B46229A134303D1079B002B00D106E3CF
:1063C000002C00DAA8E1229B1C4303D1079B002B81
:1063D00000D1A1E15B46002B00DD82E26946524616
:1063E0005346097C5C1C1170089A524500D18AE220
:1063F000310000230A22380000F08CFE0023060042
:106400000A2229003800454500D1E1E000F082FE73
:106410004146050000230A22380000F07BFEA24618
:106420008046A3E71C20069B9C4684446346069353
:10643000089B9C46844463460893049B9C46844482
:106440006346049354E74946584601F065F800282E
:1064500000DB63E7039B5946013B03930A220023B9
:10646000504600F057FE0B9B8346002B00D0CAE23B
:106470000E9B002B00DCD8E207930A9B5D460024AC
:10648000079F9B4606E0290000230A22504600F0A1
:1064900041FE050049462800FFF78AFA5B46303086
:1064A00018550134BC42EEDBAB460600079C002CBD
:1064B00000DC37E20A9B00279C46644459460122CF
:1064C000504600F0C9FF4946834601F025F80028F0
:1064D00000DC44E1651E2B780A9A06E0954200D163
:1064E000B1E0023C23782C00013D392BF6D001337A
:1064F0002B704946504600F003FE4346002B00D166
:106500002FE5002F05D0474503D03900504600F055
:10651000F7FD4146504600F0F3FD22E5130075E615
:10652000002E00D0ABE63B030024002B00D0BFE6DA
:10653000BA4B3B4200D1BBE6069B013401330693C4
:10654000049B01330493B3E601230B93239B002B9D
:1065500000DCD1E01D0098460E930793FFF7C8FBBF
:10656000079B002B00DD53E500D0ADE004980599B2
:106570000022AB4BFDF706FA3B00320001F02CFE87
:10658000002399469846002855D0239B0A9CDB435C
:1065900003934946504600F0B3FD4346002B00D11B
:1065A000DFE4B6E74A465946504600F0F5FE83461A
:1065B00053E60F9A002A00D1B6E19A4A4C46944617
:1065C000069A63440892D5E5002E00D070E6AAE74B
:1065D00000F0A0FDA24605008046C7E601239B46C9
:1065E000E2E600230B93229B022BAFD000245346FC
:1065F00021005C64504600F05BFD534618640123A3
:106600005B4207930E9302330A9023940B93ECE4BE
:10661000229B022B00DC85E6079B002BB5D1494667
:106620000522504600F076FD81460100584600F0F4
:1066300073FF0028A9DD31230A9A1370039B541CB1
:1066400001330393A5E7039B0A9A01330393312394
:1066500013704EE700230B93FFF73DFB069B5C4650
:106660009B46079B9A467CE4404602F03DFE320082
:106670003B00FDF787F900226B4BFCF773FE6B4A7A
:106680000B00944663440890099109930022644BDF
:106690003000390002F0BEFA089E099F32003B002C
:1066A00004000D0001F08EFD002800D0B2E0802033
:1066B00000068446390061440B00320020002900A6
:1066C00001F06CFD002857D00023994698465CE7FE
:1066D0000A98FFF74CFAE21A0D9BA1469C46944497
:1066E000634600240D933EE5109A119B089209938E
:1066F00002239846FFF73AFB0023524600215364D9
:10670000504600F0D5FC5346186401230A900793C5
:1067100023930E93FFF707FB43460C935B46069AC1
:10672000A846B3465546049E9146BA46002B10DD56
:1067300059460122380000F08FFE4946834600F09A
:10674000EBFE002800DC57E1392E00D122E10B9E40
:1067500031360C9B47466C1C2E709846C9E60028C3
:1067600003D1F30701D5B5E61C00631E1A78302A61
:10677000FAD0BEE6129B9946109E119F35E4012582
:10678000FFF7B4FA039B002B00D1D4E010981199C5
:106790005C420F23264A2340DB00D3181A685B684B
:1067A000FDF7F0F8241106000F00002C00D149E19C
:1067B000022398461F4D0123234209D09C462A6894
:1067C0006B6830003900E044FDF7DCF806000F008C
:1067D00064100835002CEED1FFF7E4FA039B302754
:1067E0000133039330232B70ACE45968504600F01A
:1067F0005FFC4346414604001B690C319A1C920021
:106800000C30FDF743FC01222100504600F024FE2D
:106810000C9099E50023994698460CE70000F07F1C
:10682000000014403304000000001C400000C0FCC5
:10683000C8980000A0980000129B8F49013BDB0024
:10684000C91808684968089A099BFDF79BF81490D5
:1068500015913900300002F013FD050002F044FDEF
:1068600002000B003000390002F0D4F9129B0890AE
:1068700009910A991A008C46303562444C1C0D70FF
:106880009046012B1BD008980999250000227B4BCC
:10689000FDF778F80F00060002F0F2FC040002F0A9
:1068A00023FD303402000B003000390002F0B2F951
:1068B0002C700135A845E9D14446089009911498F7
:1068C000159900226E4BFCF74DFD089A099B01F0CB
:1068D00065FC002867D0139B651E03932F780A9BE5
:1068E0002EE44346B3460C93049E069BA846994665
:1068F0005546BA46392E4DD00C9B013647466C1C86
:106900002E709846F5E54246069BB346BA46049E6D
:1069100099462F009046D1E5069B079A9B1A08934B
:10692000002327E40124C5E53623169A4C469B1A1A
:10693000069A08921EE40223109E119F9846FFF7C4
:1069400031FA079B002B00D18EE60E9C002C00DC58
:1069500012E7039B0022013B13933000474B3900A1
:10696000FDF710F8060040460F00013002F0BCFCB5
:1069700032003B00FDF706F80022424BFCF7F2FC28
:10698000414A0B009446634408900991129409937C
:10699000FFF730FA39232B700C9B47466C1C984646
:1069A0000A9A3923A1E5149A159B0020344902F074
:1069B00031F9089A099B01F005FC002801D1DBE6BA
:1069C0001C00631E1A78302AFAD0FFF7C8FA434633
:1069D000B3460C93049E069BA84699465546BA4674
:1069E000392ED7D0002C00DDB1E6B2E6139A4D4621
:1069F00003920A9BFFF7A4FB002800D0A9E6F30747
:106A000000D4A6E6A0E6002341460A22504600F044
:106A100081FB0E9B8046002B01DD079386E4229BC1
:106A2000022B1FDC0E9B079380E4229B022B19DCB8
:106A30004946FEF7BDFF0A9B303018700E9B0600DA
:106A4000079333E502239846FFF7ACF9139B149C98
:106A500003930A9B1D00FFF773FB139B149C039386
:106A6000FFF77FFA0E9B0793D6E5042B00D13FE496
:106A70003C23181AD7E4C046C89800000000244000
:106A80000000E03F00001C400000C0FC044B1B68FD
:106A9000586B002801D0F03070470248FBE7C04631
:106AA0000C0000204C080020F0B557464546DE4655
:106AB0004E46E0B50D000B3583B00700162D00D80B
:106AC0009FE007239D4300D5C4E0A94200D9C1E05F
:106AD00000F0DEFAF823FF339D4200D88FE2680A07
:106AE00000D1BBE0042800D962E138239846A80908
:106AF00080443930C100D24E71180839CC68A142A7
:106B000019D0032362689A431300521B0F2A00DD39
:106B1000AAE0002A00DB88E003239C4608E06246E6
:106B2000636893435A1B0F2A00DD9DE0002A7CDA3C
:106B3000E468A142F3D1320034690832944200D1B2
:106B400090E10323616899438946491B0F2900DDC1
:106B500062E172613261002900DB87E0B94A4B468D
:106B6000914500D930E1DB08FF3A9910FF3A8A409D
:106B7000DB0071689B190A4399687260E360A16049
:106B80009C601300CC6001218210914099426FD823
:106B90000B4205D103229043490004300B42FBD045
:106BA00003239846C3009946B144CC4682466346C7
:106BB000DC68A44507D157E1002A00DB66E1E46800
:106BC000A44500D150E14246636893435A1B0F2A03
:106BD000F2DD01208046611905436560A068E56823
:106BE0000836C560A8604046F160B1601043486057
:106BF000CE608E603800E25000F052FA200008307B
:106C000021E0102926D8380000F042FA1025182378
:106C100002208B4EF3181A005C68083A944200D1A7
:106C20002EE1032362689A431300E268A168CA60F8
:106C300091600122E318596838000A435A6000F055
:106C40002FFA2000083003B03CBC90469946A2467B
:106C5000AB46F0BD0C2300203B60F4E780213F23CE
:106C600040208900984646E7404664E74B46E0E707
:106C70000323B46862689A439046AA4203D3531B25
:106C80000F2B00DD86E0230043446F4A01936F4BD6
:106C900093461B681268EB18013200D168E16C4A18
:106CA000944663441B0B1B0300930099380000F0CB
:106CB00047FD03008146013361D0019B834200D927
:106CC000FFE0644B009A9A461B689C465346624418
:106CD0001A60019B1100834200D155E15B461B689D
:106CE000013300D16CE14B46019A9B1A5918534667
:106CF000196007234A46134000D124E10821894640
:106D00005549D21A9144CB1A009A38004A441105C9
:106D1000090D5B1A19009B4600F012FD431C00D1BF
:106D200042E14B46C01A01235844184353461B689E
:106D30005B441900534619604B46B3605860B44237
:106D400013D043460F2B00D8E8E043460722606883
:106D50000C3B9343063A024005201A436260E21856
:106D6000506090600F2B00D922E13C4B1A68914291
:106D700000D919603A4B1A68914200D9196003236F
:106D8000B46862689A43531B954200D9C9E00F2B3F
:106D900000DCC6E00122290013431143651961603C
:106DA0003800B5606B6000F07BF9200008304AE7DE
:106DB00014287AD9542800D9BAE06E239846280BB3
:106DC00080446F30C10096E65A0A042A73D9142A07
:106DD00000D9D0E011005C325B31D20008235B4265
:106DE0009C46B218944463469A6803239846944597
:106DF00000D1ABE0434651689943894500D395E003
:106E000092689445F6D16346DA6873686146E26039
:106E1000A1609460CC60B6E6012360191D436560F3
:106E200070613061C26082601A004B460A43426062
:106E30003800E15000F034F92000083003E7C04684
:106E40003C040020FF01000044080020940C0020B6
:106E50000F100000640C0020081000008C0C0020B3
:106E6000900C002073688EE608239B46073BDC44A9
:106E70009B46DA4443465246134200D097E637E039
:106E8000DC680230A34200D155E6CAE60122E318CD
:106E9000596838000A435A60E368A268D3609A6070
:106EA00000F0FEF820000830CDE65B2398468044D1
:106EB0005C30C1001FE69A09110039323831D20026
:106EC0008CE7B44200D05AE74F4B009A9A461B68B1
:106ED0009C465346624411001A60FFE608235B4259
:106EE0009C46E1444B469B680138994500D084E0BC
:106EF00043460342F2D173688B4373604900994261
:106F000000D9B5E6002900D1B2E650460B4200D0C8
:106F100048E6490004300B42FBD043E601234A46D1
:106F20005360380000F0BCF800208CE694466AE715
:106F3000AA235B00984211D8DD3B9846E80B8044B9
:106F40007830C100D7E580235B01DDE68910023B84
:106F50008B40726813437360624657E72B4B98422D
:106F60001CD87C239846A80C80447D30C100C2E523
:106F70001033009399E6542A26D84B461A0B110079
:106F80006F326E31D20029E71B0500D0A6E6012042
:106F9000009BB268434403435360E6E6FE217E2330
:106FA0007F2089009846A6E5002301209B46BDE688
:106FB00021003800083100F0E1FC53461968D4E69E
:106FC0005B464A461A6094E6AA2149008A4206D8DE
:106FD0004B46DA0B110078327731D200FEE60B49CE
:106FE0008A4206D84B469A0C11007D327C31D20081
:106FF000F4E6FE227E219200F0E673687EE72B0025
:10700000E808083305E6C046640C0020540500007B
:1070100070B5CDB2830734D0541E002A1BD003783C
:10702000AB4219D0032204E0013C14D30378AB42F5
:1070300012D001301042F7D1032C0ED8002C0AD008
:107040000378AB4208D0041902E00378AB4203D0C6
:1070500001308442F9D1002070BDFF220B061B0CC9
:10706000114019430B04084E19430368074A4B406B
:107070009A189A433242E3D1043C0430032CF4D8EA
:10708000DCE71400D8E7C04680808080FFFEFEFE6B
:1070900010B50248FDF70AF910BDC046A80D002042
:1070A00010B50248FDF704F910BDC046A80D002038
:1070B00070B50400C06C0D0000280AD0AB00C318E6
:1070C000186800280FD002681A6000230361C360AB
:1070D00070BD21220421200000F0D4FBE0640028D0
:1070E000ECD10020F4E70126AE40721D9200012190
:1070F000200000F0C7FB0028F3D045608660E4E77D
:10710000002906D04B689A00C36C9B181A680A6065
:1071100019607047F8B5CE4647468146080080B5ED
:107120000D000C691F0000211430036801311E049A
:10713000360C56431B0C5343F619370CDB19360437
:107140001F0C360C1B049B1908C08C42EDDC002F71
:1071500008D0AB689C420ADA231D9B00EB1801346F
:107160005F602C6128000CBC90469946F8BD6B68A6
:107170004846591CFFF79CFF29002B6980469A1C42
:1071800092000C310C30FCF781FF6B689A004B4683
:10719000DB6C9B181A682A601D604546DCE7C04618
:1071A0000300020C0020002A01D11B0410301A0E2B
:1071B00001D108301B021A0F01D104301B019A0FB4
:1071C00001D102309B00002B03DB01305B0000D4B7
:1071D0002020704703685A0709D00022D90704D439
:1071E0009A0720D402229B080360100070471904FC
:1071F0000022002901D11B0C1032FF21194201D1BC
:1072000008321B0A190701D104321B09990701D161
:1072100002329B08D90704D45B0801D12022E4E79D
:1072200001320360E1E75B0803600122DDE7C0464D
:1072300010B50C000121FFF73BFF012344610361FE
:1072400010BDC046F0B557464E464546DE46E0B551
:1072500014690E6985B00F001500A64204DA3300E8
:10726000170026000D001C0033199846BB6879688A
:10727000984500DD0131FFF71BFF142203009446FF
:1072800063449B4643469B005B4419000293039072
:107290005B4600228B4503D2029904C39942FCD875
:1072A0001423A4009A4614372300BC46AA44B6000F
:1072B00053440097B44401939A454FD253461B68F8
:1072C0001E04360C20D05C460027009D210008CC0F
:1072D00004CD9946484613041B0C73430004000C6C
:1072E0001B18D819130C4A467343120C9B18020C36
:1072F0009B1802041F0C120C1B0413430B60AC45BB
:10730000E4D8534627601B681E0C20D05B46002142
:107310001B685C4618000F006246009D2988000C1F
:1073200071430918C9191B0408041B0C034323608B
:1073300008CD60681B0C734307043F0CDB19090C74
:107340005B181F0C0434AA42E8D894462360042337
:107350009946019BCA44CB445345AFD84346002BC2
:107360000EDD029B043B1A68002A09D1424603E065
:10737000043B1968002902D1013A002AF8D190464D
:10738000039B424618001A6105B03CBC90469946E2
:10739000A246AB46F0BDC046F8B54746CE460323ED
:1073A00080B580460F00140013403AD1A4103E006F
:1073B000002C25D043469D6C002D3BD03E00002381
:1073C00001279946274207D1641019D02868002860
:1073D0001BD005002742F7D02A0031004046FFF7B6
:1073E00031FF002E1BD04246D26C736894469B003E
:1073F00063441A68641032601E600600002CE5D1F8
:1074000030000CBC90469946F8BD2A002900404641
:10741000FFF718FF4B46286003600500DAE7060017
:10742000D2E70B4A013B9B009A580023FFF772FEFC
:107430000700BBE701214046FFF73AFE054B050078
:107440004361012303614346986400230360B5E769
:107450009099000071020000F8B54E464546DE46A0
:107460005746E0B50E00336954119846A044434690
:107470005D1CB3688346914649689D4203DD013136
:107480005B009D42FBDC5846FFF712FE030084467A
:107490001433002C06DD0021A4001A001B1902C2BF
:1074A0009342FCD132694846970031001F221431C3
:1074B0001040CF198146002825D02022121A92466A
:1074C000002248460C688440504614431C6004C99E
:1074D0000433C2408F42F4D81A60002A01D04546D6
:1074E00002356346013D1D61736860469A005B4644
:1074F000DB6C9B181A6832601E603CBC9046994653
:10750000A246AB46F8BD04C904C38F42E9D904C9F9
:1075100004C38F42F7D8E4E70A69036930B5050070
:10752000981A11D1920014351431AB18891801E062
:107530009D4209D2043B04391C680A689442F7D082
:10754000944280410122104330BDC046F8B5454603
:10755000DE4657464E4614000B691269E0B5884670
:107560009D1A1AD10F0014218C4692001437A4449E
:10757000BB18624402E09F4200D370E0043B043A2F
:107580001E6811688E42F6D000D371E043463E007B
:10759000A04667461C00012506E0002D6ADB474631
:1075A000260000251437143643465968FFF780FD3E
:1075B00043468146C56018694D4683009C46236951
:1075C000BC449B0098460023B04414359A4600E022
:1075D000270004CE3C009346594608CC09041A04FF
:1075E000120C5244090C521A190C5B461B0CCB1A94
:1075F00011145B1812041914120C1B048A4613434D
:10760000291D2B600D00B045E2D8A44516D908CC41
:107610001A04120C524416141B0C9B1912041E144B
:10762000120C1B041343B24608C5A445EFD86246AA
:107630000324D21B053AA243043289180439002BD3
:1076400004D104390B680138002BFAD04B4618617D
:1076500048463CBC90469946A246AB46F8BD002140
:10766000FFF726FD01230361002381464361EFE715
:10767000664699E727000E00A046143714360C0022
:10768000012591E7F0B501211C0083B0089E15008B
:10769000FFF70EFD2303640007001B0B640D02D0EF
:1076A0008022520313430193002D19D068460095A0
:1076B000FFF790FD002830D1009B7B61019BBB61EF
:1076C0005A1E93415D1C3D61002C14D0194B9C4601
:1076D000352364442418181A099B3460186019E093
:1076E00001A8FFF777FD019B20307B610123012575
:1076F0003B61002CEAD1104B9C46104B6044EB18C8
:107700009B00FB1830605869FFF74AFD6B01181A9F
:10771000099B1860380003B0F0BD019B20221900BE
:10772000121A91400A00C340009901930A437A61FA
:10773000C5E7C046CDFBFFFFCEFBFFFFFFFFFF3FCE
:10774000002370B5064C050008002360FBF726F8FF
:10775000431C00D070BD2368002BFBD02B60F9E7E1
:10776000BC0D0020F0B557464E46DE464546E0B516
:10777000936883B001900E009246002B70D08D6804
:1077800013682C0008681D0046E09022B389D200DF
:10779000134230D03169421A934670694200121880
:1077A000D00F8218521090465A46501CC0194246BB
:1077B000404501D9804602008020C000034238D0F5
:1077C00011000198FFF770F9041E54D05A46316930
:1077D000FCF75CFCB3892A4A134080221343B3812F
:1077E000434620005A463461B8463C005844736111
:1077F0009B1A3060B3604246494600F0B3F9B36863
:107800001C1B3368B46043443360180053469B68C4
:10781000DF1B53469F6023D06F682B000835002F75
:10782000FAD01B68A0469946A742AED23C00B846A3
:10783000E1E7019800F0E6F9041ED1D1019C31691D
:10784000200000F09BF80C2323604022B389012024
:107850001343B3815246002340429360536003E0D8
:10786000002352460020536003B03CBC904699462A
:10787000A246AB46F0BD0C23019A1360E5E7C04673
:107880007FFBFFFF10B55143FFF70EF9041E1CD01C
:107890000300083B5A6803239A43043A242A16D863
:1078A0000300132A0DD900210833016041601B2A0F
:1078B00007D98160C160242A0DD10300016118330A
:1078C000416100221A605A609A60200010BD0021B8
:1078D000FCF71EFCF9E703001033F2E7F8B50C00E3
:1078E0000600FFF7D5FB204FBB685D6803239D436F
:1078F0001E4B2C1B9C466444240B1D4B013C240353
:107900009C4207DD00213000FFF71AFFBB685B19BE
:10791000984204D03000FFF7C3FB0020F8BD61425D
:107920003000FFF70DFF431C0DD00122BB682D1B5B
:1079300015435D600F4B30001A68141B1C60FFF785
:10794000AFFB0120EAE700213000FFF7F9FEBA683B
:10795000831A0F2BDEDD08490968401A05490860C3
:1079600001210B435360D5E73C040020EF0F0000DA
:10797000FF0F0000640C002044080020F8B504004C
:107980000D1E3CD0FFF784FB29000839486801230D
:10799000050003269D434A199C46614F5368B34333
:1079A000BE68B24256D06646536006420AD13E00D7
:1079B00008680836091A2D188868B04265D0CE6864
:1079C000C660B0600120D6187668064233D0554BA9
:1079D000284348604D519D4212D8ED08FF3BAA1044
:1079E000FF3B93407A68ED0013437B60EF19BB685F
:1079F000CF608B60B960D9602000FFF751FBF8BD04
:107A0000680A042850D8A809020039303832C0006A
:107A1000381808388368032698424CD05A68B24315
:107A2000954230D29B689842F8D1C368CB60886099
:107A30009960C160E0E7ED183B4E9368B34242D0D5
:107A4000D2682843DA609360364B48604D519D42BE
:107A5000D6D8C2E76246EB18024206D10A68891AF4
:107A600088689B18CA68C260906001221A434A6005
:107A70002E4AB96012689342BED32D4B200019687C
:107A8000FFF72CFFB8E71800CFE76646D01840682C
:107A900030423FD190685D19D368C36098606346F7
:107AA0002B434B604D51A7E7142814D802005C30DB
:107AB0005B32C000ACE70123921093407A68134315
:107AC0007B600300B2E72843D9609960CB608B608C
:107AD00048604D5190E7542805D8280B02006F30BC
:107AE0006E32C00094E7AA225200904205D8E80BFB
:107AF000020078307732C0008AE70E4A904205D8FB
:107B0000A80C02007D307C32C00081E7FE207E227E
:107B100080007DE763462B434B6015606CE7C046F1
:107B20003C040020FF01000044040020480800201D
:107B3000940C00205405000082B000290AD0002ACD
:107B40000BD0002B0BD013780B601078431E98419C
:107B500002B0704701A9002AF3D10020F8E7022003
:107B60004042F5E7F0B588420AD98B18984207D20F
:107B7000531E002A03D0CA5CC254013BFBD2F0BDA5
:107B800005000F2A08D8002AF9D00023CC5CEC5459
:107B900001339342FAD1F2E70B0003439B072DD147
:107BA00015000C000300103D2F0901373F01C719D4
:107BB00026681E6066685E60A6689E60E66810348F
:107BC000DE6010339F42F3D10F24A54310354919CD
:107BD00014404519032C13D90023271FBE08013672
:107BE000B600CC58EC500433B342FAD10326B74365
:107BF0003C1D09192D193240C7D1C0E70500C4E763
:107C00002200C0E7F0B54E464546DE465746E0B591
:107C100085B001900E001500002900D19EE03700CC
:107C20000198083FFFF734FA7A68032314009C4355
:107C30002B000B33B946162B47D81021102388464A
:107C4000454546D89C4249DACC4938198B46896863
:107C50000290884200D1C2E001218A4640680100BA
:107C60000390504681438C4602998B46DC44614622
:107C7000496801424DD0104200D1A2E0290001988C
:107C8000FEF712FF051E39D0012302007968083A79
:107C900099437F18BA4200D12EE1221F242A00D92D
:107CA00014E1132A00D9E8E00300320011681960DA
:107CB0005168596092689A60019C31002000FFF77A
:107CC0005DFE2000FFF7ECF91BE007218B4398468F
:107CD000B6D50C23019A0025136012E03500434607
:107CE000E31A0F2B25D84B46012249465B68134007
:107CF00023434B604C4463681A4362600198FFF76A
:107D0000CFF9280005B03CBC90469946A246AB4648
:107D1000F0BD032103988C46884321188B46994275
:107D200021DB029A3500D36892685C46D3609A6082
:107D3000D5E74A460120464652684946024032434A
:107D40004E464144034372604C444B6063680831C3
:107D5000184360600198FFF711FECFE71100FEF7AE
:107D6000A3FE0500CDE75146114200D086E76146EB
:107D70003A68BA1A924652688A4380188346A344E6
:107D80009B4526DB029AD3689268D3609A6053467B
:107D9000524655469268DB680835D3609A60221FC8
:107DA000242A00D996E0132A72D953463168996083
:107DB0007168D9601B2A00D9A4E032001033083260
:107DC00068E03A68BA1A92465146032249689143DC
:107DD0000A009346A3449B4500DA4FE7D7E7032008
:107DE000029984464968814340460919103002903F
:107DF000814258DAD20700D540E760463A68BA1A9D
:107E00009246526882430298511803918842E0DCFE
:107E10005346524655469268DB680835D3609A60EF
:107E2000221F242A00D98EE0132A00D888E0534666
:107E3000316899607168D9601B2A00D988E03200E6
:107E400010330832116819605168596092689A605D
:107E500051465B46424641449960039B01989A1AF9
:107E600001231A434A605246526813404246134364
:107E700052465360FFF714F943E7336803607368B1
:107E800043601B2A2DD803003200083308320DE767
:107E90002B00320011685C4619605168D146596068
:107EA00092689A601BE74346FA185B469A6043461D
:107EB000C91A0123194351607A6801981340424658
:107EC00013437B60FFF7ECF835001AE73100FFF74A
:107ED00049FEF1E631002800FFF744FE5C46D1463A
:107EE000FDE6B3688360F368C360242A15D00300FD
:107EF000320010331032D9E6536803229343E4185A
:107F00003500ECE65346B1681961F1685961242ADD
:107F10000CD0320018331032BCE7336932000361F1
:107F200003007169183318324161BFE65346326964
:107F300051469A613200706920331832C861A9E74E
:107F40002B0032007EE731002800FFF70BFE7FE7B1
:107F50005346B1681961F1685961242A03D032008F
:107F6000183310326EE75346326951469A61320037
:107F7000706920331832C86164E7C0463C040020B1
:107F8000002904D0FF2A04D801200A70704700207D
:107F9000FCE78A23036001204042F7E703460B43D6
:107FA0007FD4002243088B4274D303098B425FD3F2
:107FB000030A8B4244D3030B8B4228D3030C8B421E
:107FC0000DD3FF22090212BA030C8B4202D3121204
:107FD000090265D0030B8B4219D300E0090AC30BD9
:107FE0008B4201D3CB03C01A5241830B8B4201D386
:107FF0008B03C01A5241430B8B4201D34B03C01A6F
:108000005241030B8B4201D30B03C01A5241C30AE6
:108010008B4201D3CB02C01A5241830A8B4201D357
:108020008B02C01A5241430A8B4201D34B02C01A41
:108030005241030A8B4201D30B02C01A5241CDD2E6
:10804000C3098B4201D3CB01C01A524183098B4231
:1080500001D38B01C01A524143098B4201D34B011A
:10806000C01A524103098B4201D30B01C01A52417D
:10807000C3088B4201D3CB00C01A524183088B4204
:1080800001D38B00C01A524143088B4201D34B00ED
:10809000C01A5241411A00D201465241104670475F
:1080A0005DE0CA0F00D04942031000D34042534064
:1080B00000229C4603098B422DD3030A8B4212D324
:1080C000FC22890112BA030A8B420CD38901921156
:1080D0008B4208D3890192118B4204D389013AD093
:1080E000921100E08909C3098B4201D3CB01C01A68
:1080F000524183098B4201D38B01C01A524143097B
:108100008B4201D34B01C01A524103098B4201D368
:108110000B01C01A5241C3088B4201D3CB00C01AD5
:10812000524183088B4201D38B00C01A5241D9D2ED
:1081300043088B4201D34B00C01A5241411A00D26E
:108140000146634652415B10104601D34042002B6A
:1081500000D54942704763465B1000D3404201B5E9
:108160000020FAF7FFFB02BD0029F8D016E77047A0
:108170008446101C62468C46191C634600E0C046CB
:108180001FB500F0E5FC002801D40021C8421FBD46
:1081900010B500F03FFC4042013010BD10B500F0BA
:1081A000D7FC002801DB002010BD012010BDC04617
:1081B00010B500F0CDFC002801DD002010BD01202D
:1081C00010BDC04610B500F05FFC002801DC0020A7
:1081D00010BD012010BDC04610B500F055FC0028B0
:1081E00001DA002010BD012010BDC046002B11D1C6
:1081F000002A0FD1002900D1002802D00021C94354
:10820000081C07B4024802A14018029003BDC046F2
:1082100055A7FFFF03B4684601B5029800F006F8C1
:10822000019B9E4602B00CBC7047C046F0B5574655
:108230004E464546DE46E0B5040083B00D0092464A
:1082400099468B422FD82CD04946504601F08EF8E3
:1082500029000600200001F089F8331A9846203BD7
:108260009B4600D574E053465A4693401F00534640
:10827000424693401E00AF4229D826D05B46A41B3D
:10828000BD41002B00DA79E0002200230092019327
:1082900001235A46934001930123424693400093A1
:1082A00019E08242D0D900220023009201930C9B56
:1082B000002B01D01C605D600098019903B03CBCAC
:1082C00090469946A246AB46F0BDA342D6D90022BD
:1082D0000023009201934346002BE8D0FB0772086D
:1082E0001A4346467B080EE0AB4201D1A2420CD8AD
:1082F000A41A9D41012024196D410021013E24183A
:108300004D41002E06D0AB42EED9013E24196D41FD
:10831000002EF8D15B460098019900196941002BA5
:1083200022DB2B005A46D3402A004446E2401C0080
:108330005B461500002B2CDB26009E4033002600F8
:108340004746BE403200801A994100900191AEE745
:10835000424620239B1A5246DA40414613004A46C1
:108360008A4017001F4382E7424620239B1A2A00B7
:1083700046469A402300F3401343D5E74246202364
:1083800000219B1A0022009101920122DA40019201
:1083900082E74246202326009B1ADE402F00B44687
:1083A000974066463B003343C9E7C046F0B55746A1
:1083B0004546DE464E46E0B54C000E0387B0834688
:1083C00092461D008046360B640DCF0F002C4FD017
:1083D0006F4B9C4235D08023420F1B04F6001343A1
:1083E00033439946C30098466A4B00269C460023B7
:1083F000644403932B031B0B9B466B00ED0F50460D
:108400005B0D01955ED0624A934253D05A46D1002B
:108410008022400F120402430A4393465246D10081
:108420005C4A9446002263443800684084460290C7
:10843000E41A16430F2E00D9B4E0574BB6009B59EF
:108440009F460300334399466CD10023984602337C
:1084500008260393CEE7CB464146039A0197022AAA
:1084600065D1019B4A4C9C460023002298466BE054
:108470000300334399464ED0002E00D1BCE13000BA
:10848000FBF7C2FD03000B3B1C2B00DDACE11D2202
:10849000D31A5A460100DA4008398E40130033439C
:1084A00099465B468B40984600233C4C0026241A94
:1084B00003939FE751465A46114329D10022934620
:1084C0000232B1E7594601431ED05B46002B00D172
:1084D0009EE15846FBF798FD03000B3B1C2B00DD8B
:1084E0008FE102005946083A91408B461D21CB1A74
:1084F0005146D9400B0059460B4351469B4691408B
:10850000264B00221B1A8FE7002301229B468BE794
:108510005146032288E700239846013304260024AD
:10852000039367E70323B14603930C2662E7032A0C
:1085300000D15CE2019B012A00D0E4E113409C469B
:10854000002300240022984600211203130B0A0D79
:1085500012051A432305124C40462240134362463B
:108560005B00D2075B081343190007B03CBC904680
:108570009946A246AB46F0BD002380229C461203DA
:108580009846034CE0E70023014C00229846DBE7C5
:10859000FF07000001FCFFFFB09A00000DFCFFFF89
:1085A000FFFF0F80D94500D939E100D134E1002324
:1085B00046464D469A46013C5B460A0E1B021A434C
:1085C0000B02170C039313041B0C39002800904670
:1085D0000193FAF73DF90200019B83465A432800B4
:1085E00039009146FAF7BAF9350C09040D43A9454B
:1085F0000DD95B464544013BA84500D93AE1A94560
:1086000000D837E102235B429C464544E3444B4695
:10861000EB1A390018000493FAF71AF9019B0500C8
:108620004343390004989946FAF798F9330409044A
:108630001B0C0B43994509D943446A1E984500D940
:108640001AE1994500D817E1023D43444A469B1A76
:108650005A4612042A4303999346100C0A0C914679
:1086600009045A46090C4E460D001204120C4543EB
:10867000059151437243704352190E0CB218954242
:1086800003D980256D02AC466044150C0904120420
:10869000090C28185218834200D2CEE000D1C8E05D
:1086A0001D1A53469E1AB24592415242AB1A9A463F
:1086B000984500D117E139001800FAF7C9F8019B75
:1086C00005004343390050460493FAF747F90498EC
:1086D0000B04310C1943884209D941446B1E88456B
:1086E00000D907E1884200D804E1023D4144049BDF
:1086F000CB1A180039000493FAF7AAF8019B8246B6
:108700004343390004980193FAF728F901980B04C0
:108710003104090C194388420DD953464144013BA9
:10872000884500D9E8E0884200D8E5E002235B42B2
:108730009C464144E244019B2D04CE1A51462943F4
:10874000059D4F462A000B04080C1B0C5A43454359
:108750007B4378435B19170CFB189D4203D9802596
:108760006D02AC4660441D0C12041B04120C281848
:108770009B18864200D293E000D18EE0012319437A
:10878000A04BE318002B00DC99E04A0700D09EE0E4
:108790005A46D20106D55A469B4B1A40802393462F
:1087A000DB00E318994A934268DD0123029A984C52
:1087B0001A400023944698460022C5E680224B4684
:1087C000120313420AD05B46134206D11A43120326
:1087D000120BAC4688468E4CB6E64B461A43120343
:1087E000120BBC468A4CAFE603005A46283B9A401F
:1087F00000239146984657E65846FBF705FC203083
:1088000040E603005246283B9A400021934677E613
:10881000FBF7FAFB20305FE6884500D2C7E64B46FF
:10882000DE075D0843465B081E434346DB079A4666
:10883000C2E60025924500D333E7039E5946B4466D
:10884000E244B245AD416D424544EB1801399845CB
:1088500007D2984200D97FE000D1BCE01D1A8B46B8
:108860001FE79845FAD1039D5545F2D943468B46FB
:108870001D1A16E79B46CAE61500E7E65A46C908E0
:1088800052070A435B0590465C0D5A460123029944
:1088900052021940120B8C4656E6002B00D16FE7AE
:1088A00046444A1EB04529D91100864200D065E7EA
:1088B000039A934200D061E762E701214942012017
:1088C000C21A382A21DD029B03409C4638E60F225B
:1088D0000A40042A00D15BE70A00111D914292412F
:1088E0005242934454E7474BE318002BE5DD012245
:1088F0005242F2E71D00FAE69A461CE7B04239D828
:108900006ED011003AE702933AE71F2A3CDC20239D
:108910009B1A0C005846994098404B1E99415B4663
:10892000D440D340204308431A00430709D00F2303
:108930000340042B05D00100081D88429B415B4287
:10894000D21813023AD50123029A01241A400023B7
:10895000944698460022F7E5022149428C46039D41
:10896000E344AC46E244AA45AD416D424544ED18AE
:108970002D1A96E68A1E03994D008D42894149427F
:108980004144761803958FE71F204042C31A58468A
:10899000D8400300202A28D040205D46821A954006
:1089A00029434A1E91411943072300220B4009D055
:1089B0000F2300220B400800042BBDD101005307F8
:1089C0005202120BC9081943012388460299002458
:1089D00019408C46B8E55245BED88B46002560E666
:1089E000039D9D42C6D3110062E70025D8E780228F
:1089F0005B4612031A43019B1203120B9C468846E6
:108A0000034CA1E5FF030000FFFFFFFEFE0700008F
:108A1000FF070000F0B54F464646D6465C00C0B59D
:108A20001F03DB0F9A46174B0E034D00844680460A
:108A3000360B6D0DC90F91463F0B640D01209D4211
:108A400008D09C4201D0A5420BD01CBC9046994650
:108A5000A246F0BD63463343F7D1AC42F5D13A4369
:108A6000F3D10120BE42F0D1C845EED1514507D027
:108A7000002DEAD163461E433000461EB041E4E7B4
:108A80000020E2E7FF070000F0B54546DE46574606
:108A90004E46E0B51F033D0B2C4F0E034C00AB467A
:108AA0005D008446360B640DC90F90466D0DDB0FDB
:108AB000BC422AD0254FBD422DD0002C0FD13043CF
:108AC0000700814678427841C0B2002D17D15F4639
:108AD0003A4314D14B460020002B0AD006E0002D6B
:108AE00002D15846024301D0994218D04842012190
:108AF00008433CBC90469946A246AB46F0BD0028D0
:108B0000F2D00120013B1843F3E737000743D1D0EF
:108B100002204042EDE75F461743CED0F8E7AC4273
:108B2000E4DC03DA481E01210843E2E75E45DDD8B4
:108B300006D000205E45DCD20123481E1843D8E74A
:108B4000C445D3D80020C445F6D3D2E7FF070000C0
:108B5000F0B54E464546DE4657465C00E0B51F037D
:108B6000DB0F99462A4B0E034D00C90F8446360B86
:108B70006D0D8B4690463F0B640D9D4220D0244BDB
:108B80009C4222D0002D12D1304343424341DBB2FC
:108B9000002C1FD0002B0CD04B460120013B03437F
:108BA00018003CBC90469946A246AB46F0BD002C4E
:108BB00016D0CB4517D05B46594201230B43EFE754
:108BC000310002230143EBD1D9E7390002231143DD
:108BD000E6D1D7E73A43DDD100230028E0D0EAE729
:108BE0003A43E6D1E7E7A542E5DC05DBBE42E2D841
:108BF00007D00023BE42D3D25946012301390B438B
:108C0000CEE7C445D7D80023C445F5D3C8E7C0464E
:108C1000FF070000F0B54646D6464F460C03C0B5E8
:108C2000CD0F4E00610A440F0C43C1005800400DA7
:108C300084468A460F001903500F490A0143C6486B
:108C4000760DA846DB0FD200844500D1D8E0012084
:108C50004340AB4200D1A6E06046351A002D00DC4F
:108C600005E1002810D10B00134300D1D7E06B1EA3
:108C7000002B00D04BE153469F1ABA458041641A3D
:108C80004042241A01261EE0B34B9E4248D0802366
:108C90001B041943382D00DD19E11F2D00DD4CE1C7
:108CA00020230F005B1B10009A409F40E840531E9A
:108CB0009A41E940074317435346DF1B611ABA45FF
:108CC000A44164420C1B230200D4C5E06402650A7F
:108CD000002D00D1F6E02800FBF796F90300083BD1
:108CE0001F2B00DDE9E020223C00D21A9D40D44039
:108CF0009F4025439E4200DDDBE09E1B731C1F2B23
:108D000000DD0AE120223800D21A290097402C0009
:108D10009140D8407A1E9741DC40002601430F4322
:108D20007B0709D00F233B40042B05D03B1DBB42E2
:108D3000BF417F42E4191F00230225D5864B01362F
:108D40009E4200D1AFE0854B01251C40434662079F
:108D5000FF08640276051743240B760D1D400021A1
:108D60002403230B0C0D7E4A24051C4314403305B9
:108D700023435B00ED075B082B43380019001CBC44
:108D800090469946A246F0BD012543466207FF087A
:108D90001743E4081D40704B9E4236D024037605ED
:108DA000240B760DDBE76346F31A002B00DC94E01E
:108DB0006046002835D068488642B1D080273F04FD
:108DC0003943382B00DCFDE00A43170000217A1EEE
:108DD0009741574457458041091944420C192302D1
:108DE0003AD55D4B01369E4200D14BE101225B4BEF
:108DF0001C407B0817401F43E207174364088FE7B6
:108E00000800104300D024E721E723003B4300D1B2
:108E1000B9E18022120314432403240B9FE72E00A0
:108E20007EE70800104300D1CAE0581E844600289F
:108E300000D0E7E052445245804164184042241873
:108E400017000126230207D50226CFE764462C43EC
:108E500000D1B3E12C0067467B0700D062E76307CF
:108E6000FF081F4301254346E4081D4093E7002DFA
:108E700078D1751C6D056D0D012D00DCF2E05046BA
:108E8000801A8245BF41651A7F42ED1B8446280245
:108E900000D48CE05046171ABA4292410C1B55423E
:108EA000651B984614E70125434600241D40002712
:108EB00055E72A4CF61A2C4032E73D002838854009
:108EC000002717E73800FBF79FF8203006E70A4332
:108ED000170000217A1E9741EEE6002B00D0E5E056
:108EE000731C9C465B055B0D012B00DC9FE01A4B5D
:108EF0009C4500D1C5E0524452458041641840422F
:108F00002418E707520817436408664608E7124822
:108F1000854200D185E01D00BCE629001F3EF140DE
:108F2000202B00D17FE04022D31A9D402F437D1E8D
:108F3000AF4100240F4300268EE72B000F00203B9B
:108F4000DF40202D71D040235D1BA9400A43511EF4
:108F50008A4100211743AFE6FF070000FFFF7FFFB4
:108F6000FFFF0F80002E3ED0B34EB44545D0802683
:108F700036046D423443382D00DDA8E01F2D00DD9E
:108F80001FE1202627005046761BB740E8400743E4
:108F90005046B040461EB041EC403843171ABA4222
:108FA00092410C1B5242A41A664698468BE66446D0
:108FB00067462C4300D08BE6002500260027EAE612
:108FC0001E00ADE61F2B60DC2027F81A0F00844638
:108FD00087401000D840074360468240501E8241BF
:108FE000D9401743F5E626005046064305D0ED4329
:108FF000002DD3D0904EB445BDD10C00170066466D
:1090000098468DE68C4883420BD06346D9E6002D06
:1090100000D096E00800104300D1E2E00C001700F9
:109020009846854E7CE6002580E700218EE72300E8
:1090300050460343002E00D0A8E0002B00D1DEE014
:109040000B00134300D16BE6524452458041641833
:10905000404224181700230200D4FDE6774B6646F1
:109060001C405DE6250050460543002ECFD1002D63
:109070004FD10C00144300D1A0E00C00170098461B
:109080004EE666460024002785E61F000800203FC4
:10909000F8400700202B00D18EE04020C31A9940F1
:1090A0000A43511E8A410021174392E6002E14D133
:1090B00026005046064362D0DB43002B5CD1871864
:1090C0009742924164185242A418664687E6504679
:1090D0002043441EA041002460E7574EB4454ED0C3
:1090E000802636045B423443382B00DD7FE01F2BA3
:1090F00000DD8BE0202627005046F61AB740D84006
:1091000007435046B040461EB0410743DC40BF18FD
:10911000D6E70D00154300D102E65046801A82457D
:10912000BF41651A7F42ED1B8446280200D48DE6BC
:109130005046171ABA4292410C1B5242A41A984642
:10914000EEE50D00154300D16BE750466707C008F8
:1091500007438020E4080003044207D0CD080542FD
:1091600004D12C009846D70849070F437B0FE40031
:109170001C43FF00304ED3E52F4EB445B4D10C0054
:1091800017006646CCE500270024E8E5002B39D01F
:109190000B00134300D144E7C00867070743802052
:1091A000E40800030442E1D0CB080342DED1D70833
:1091B00049070F431C00D9E7002171E7002500276C
:1091C000E9E52E002700203EF740202D2FD0402635
:1091D000751BAC4050462043441EA0410024384338
:1091E000DCE6802400252403134E0027D3E55046F7
:1091F00020430700781E87410024BF1860E70C0059
:1092000017008DE50C0017000B4E89E51E002700A6
:10921000203EF740202B0CD04026F31A9C405046AD
:109220002043441EA04107430024BF1848E7002400
:10923000D0E70024F3E7C046FF070000FFFF7FFFF1
:1092400070B50E4E0D031C0349005B002D0B490D3C
:10925000240B5B0DB14204D0084900208B4208D09A
:1092600070BD05430120002DFAD1044900208B4236
:10927000F6D114432000441EA041F1E7FF0700008F
:1092800030B5134D0A034B00120B5B0DC90F0024C0
:10929000AB4210DD0F4CA3420FDC80240E4D640363
:1092A0002243ED1A1F2D0BDD0C48C31ADA4054423D
:1092B000002900D11400200030BD094BCC18FAE77A
:1092C000084CE840A44663449A400243EFE7C04696
:1092D000FE0300001D04000033040000130400001E
:1092E000FFFFFF7FEDFBFFFF70B5002830D0C317F5
:1092F000C4185C40C50F2000FAF786FE174B184AC9
:109300001B1AD21A1F2A18DD164AD21A94400022BC
:1093100024035B05240B5B0D0021100024030A0DC0
:10932000240B12052243104C1B05224013435B0003
:10933000ED075B082B43190070BD210091400A0026
:109340000B21081AC4405B052403240B5B0DE3E7E3
:109350000025002300240022DEE7C0461E04000092
:109360003304000013040000FFFF0F8010B5002934
:1093700003D1FAF749FE203002E0081CFAF744FE58
:1093800010BDC046260300007205000072050000F3
:1093900072050000720500007205000072050000F1
:1093A00072050000720500007205000072050000E1
:1093B00072050000720500007205000072050000D1
:1093C000720500000E030000720500007205000027
:1093D00072050000720500007205000072050000B1
:1093E00072050000720500007205000072050000A1
:1093F0007205000072050000720500007205000091
:10940000720500001E0300007205000072050000D6
:109410007205000072050000720500007205000070
:109420007205000072050000720500007205000060
:109430007205000072050000720500007205000050
:1094400072050000160300002E030000F602000063
:1094500006030000FE0200000200000003000000FE
:1094600028000000290000000400000005000000A2
:10947000060000000700000020000000210000009E
:10948000220000002300000024000000250000004E
:10949000260000002700000008000000090000006E
:1094A0000A0000000B00000000080042000C00420F
:1094B000001000420014004200180042001C00424C
:1094C00050756C73652077696474683A2025640A66
:1094D0000000000000010000000200000004000085
:1094E000040202001A1A1B00FFFFFF00FFFFFF002B
:1094F000FFFF00000804020001000000020000005D
:10950000040000000800000000100000002000001F
:109510000040000000800000000001000000020088
:109520000000040000000800476F696E6720666F46
:109530007277617264210A00476F696E6720626109
:10954000636B7761726473210A00000053746F705B
:1095500070696E67210A000025630000555341526F
:109560005420446562756767696E6720696E697427
:1095700069616C697A65640A0000000026210000B8
:109580002221000022210000882100008821000003
:109590003A2100002C21000040210000762100002B
:1095A00010220000F0210000F02100007C220000C9
:1095B000022200001E220000F42100002C220000E4
:1095C0006C220000B42E0000842E0000962E0000B5
:1095D000D82D0000962E00007A2E0000962E000056
:1095E000D82D0000842E0000842E00007A2E00006A
:1095F000D82D0000E02D0000E02D0000E02D00003F
:109600009C2E0000842E0000842E0000582E0000A6
:109610003C2F0000582E00007A2E0000582E00002B
:109620003C2F0000842E0000842E00007A2E0000C3
:109630003C2F0000E02D0000E02D0000E02D000098
:10964000462F0000E43000003430000034300000C9
:1096500032300000D6300000D6300000CC300000A0
:1096600032300000D6300000CC300000D630000090
:1096700032300000DC300000DC300000DC30000064
:109680006C310000743B0000343A0000343A0000B2
:10969000303A00004C3B00004C3B00003E3B0000D9
:1096A000303A00004C3B00003E3B00004C3B0000C9
:1096B000303A0000543B0000543B0000543B000093
:1096C000583D0000100000201049000084490000AF
:1096D00084490000F44800008449000084490000E7
:1096E0008449000084490000844900008449000046
:1096F000FC480000DE43000084490000984300005D
:10970000E843000084490000344400001E46000085
:109710001E4600001E4600001E4600001E460000B9
:109720001E4600001E4600001E4600001E460000A9
:1097300084490000844900008449000084490000F5
:1097400084490000844900008449000084490000E5
:1097500084490000844900003C4400008445000026
:1097600084490000844500008449000084490000C9
:1097700084490000844900004E46000084490000EE
:1097800084490000564600008449000084490000D6
:10979000844900008449000084490000F846000024
:1097A00084490000844900002A47000084490000E1
:1097B0008449000084490000844900008449000075
:1097C0008449000084490000844900008449000065
:1097D00084490000244800005848000084450000E7
:1097E00084450000844500006A4800005848000095
:1097F0008449000084490000724800008449000048
:109800008C47000052490000C8480000C2470000D1
:1098100084490000CA470000844900002049000034
:10982000844900008449000082480000494E4600F7
:10983000696E66004E414E006E616E00303132330B
:10984000343536373839414243444546000000003C
:1098500030313233343536373839616263646566A6
:1098600000000000286E756C6C29000030000000BC
:1098700020202020202020202020202020202020E8
:1098800030303030303030303030303030303030D8
:10989000496E66696E697479000000004E614E0081
:1098A0000080E03779C34143176E05B5B5B89346DC
:1098B000F5F93FE9034F384D321D30F94877825AA8
:1098C0003CBF737FDD4F1575000000000000F03FC6
:1098D000000000000000244000000000000059408B
:1098E0000000000000408F40000000000088C340DE
:1098F00000000000006AF8400000000080842E4153
:1099000000000000D01263410000000084D797419E
:109910000000000065CDCD41000000205FA00242A4
:10992000000000E876483742000000A2941A6D4219
:10993000000040E59C30A2420000901EC4BCD6420C
:1099400000003426F56B0C430080E03779C34143B7
:1099500000A0D8855734764300C84E676DC1AB432D
:10996000003D9160E458E143408CB5781DAF15444B
:1099700050EFE2D6E41A4B4492D54D06CFF0804426
:10998000F64AE1C7022DB544B49DD9794378EA443B
:1099900005000000190000007D00000043000000E9
:1099A000504F5349580000002E0000000020202096
:1099B000202020202020282828282820202020207F
:1099C000202020202020202020202020208810104F
:1099D00010101010101010101010101010040404AB
:1099E0000404040404040410101010101010414169
:1099F0004141414101010101010101010101010157
:109A0000010101010101010110101010101042426A
:109A10004242424202020202020202020202020226
:109A200002020202020202021010101020000000C6
:109A30000000000000000000000000000000000026
:109A40000000000000000000000000000000000016
:109A50000000000000000000000000000000000006
:109A600000000000000000000000000000000000F6
:109A700000000000000000000000000000000000E6
:109A800000000000000000000000000000000000D6
:109A900000000000000000000000000000000000C6
:109AA00000000000000000000000000000000000B6
:109AB000A485000086850000408500005E840000CB
:109AC0004085000078850000408500005E8400002D
:109AD0008685000086850000788500005E84000091
:109AE000568400005684000056840000BC870000A5
:109AF000F8B5C046F8BC08BC9E467047514200000D
:109B0000DD000000F8B5C046F8BC08BC9E467047B2
:049B1000B50000009C
:089B140018E7FF7F01000000CB
:109B1C00401F0000080000000100000010000020A1
:109B2C0000000000FC02002064030020CC03002095
:109B3C000000000000000000000000000000000019
:109B4C000000000000000000000000000000000009
:109B5C0000000000000000000000000000000000F9
:109B6C0000000000000000000000000000000000E9
:109B7C0000000000000000000000000000000000D9
:109B8C0000000000000000000000000000000000C9
:109B9C0000000000000000000000000000000000B9
:109BAC0000000000000000000000000000000000A9
:109BBC000000000000000000000000000000000099
:109BCC000000000000000000010000000000000088
:109BDC000E33CDAB34126DE6ECDE05000B0000004D
:109BEC000000000000000000000000000000000069
:109BFC000000000000000000000000000000000059
:109C0C000000000000000000000000000000000048
:109C1C000000000000000000000000000000000038
:109F4C000000000000000000980D00200000000040
:109F5C00000000003C0400203C04002044040020CD
:109F6C00440400204C0400204C0400205404002025
:109F7C00540400205C0400205C04002064040020D5
:109F8C00640400206C0400206C0400207404002085
:109F9C00740400207C0400207C0400208404002035
:109FAC00840400208C0400208C04002094040020E5
:109FBC00940400209C0400209C040020A404002095
:109FCC00A4040020AC040020AC040020B404002045
:109FDC00B4040020BC040020BC040020C4040020F5
:109FEC00C4040020CC040020CC040020D4040020A5
:109FFC00D4040020DC040020DC040020E404002055
:10A00C00E4040020EC040020EC040020F404002004
:10A01C00F4040020FC040020FC04002004050020B3
:10A02C00040500200C0500200C0500201405002060
:10A03C00140500201C0500201C0500202405002010
:10A04C00240500202C0500202C05002034050020C0
:10A05C00340500203C0500203C0500204405002070
:10A06C00440500204C0500204C0500205405002020
:10A07C00540500205C0500205C05002064050020D0
:10A08C00640500206C0500206C0500207405002080
:10A09C00740500207C0500207C0500208405002030
:10A0AC00840500208C0500208C05002094050020E0
:10A0BC00940500209C0500209C050020A405002090
:10A0CC00A4050020AC050020AC050020B405002040
:10A0DC00B4050020BC050020BC050020C4050020F0
:10A0EC00C4050020CC050020CC050020D4050020A0
:10A0FC00D4050020DC050020DC050020E405002050
:10A10C00E4050020EC050020EC050020F4050020FF
:10A11C00F4050020FC050020FC05002004060020AE
:10A12C00040600200C0600200C060020140600205B
:10A13C00140600201C0600201C060020240600200B
:10A14C00240600202C0600202C06002034060020BB
:10A15C00340600203C0600203C060020440600206B
:10A16C00440600204C0600204C060020540600201B
:10A17C00540600205C0600205C06002064060020CB
:10A18C00640600206C0600206C060020740600207B
:10A19C00740600207C0600207C060020840600202B
:10A1AC00840600208C0600208C06002094060020DB
:10A1BC00940600209C0600209C060020A40600208B
:10A1CC00A4060020AC060020AC060020B40600203B
:10A1DC00B4060020BC060020BC060020C4060020EB
:10A1EC00C4060020CC060020CC060020D40600209B
:10A1FC00D4060020DC060020DC060020E40600204B
:10A20C00E4060020EC060020EC060020F4060020FA
:10A21C00F4060020FC060020FC06002004070020A9
:10A22C00040700200C0700200C0700201407002056
:10A23C00140700201C0700201C0700202407002006
:10A24C00240700202C0700202C07002034070020B6
:10A25C00340700203C0700203C0700204407002066
:10A26C00440700204C0700204C0700205407002016
:10A27C00540700205C0700205C07002064070020C6
:10A28C00640700206C0700206C0700207407002076
:10A29C00740700207C0700207C0700208407002026
:10A2AC00840700208C0700208C07002094070020D6
:10A2BC00940700209C0700209C070020A407002086
:10A2CC00A4070020AC070020AC070020B407002036
:10A2DC00B4070020BC070020BC070020C4070020E6
:10A2EC00C4070020CC070020CC070020D407002096
:10A2FC00D4070020DC070020DC070020E407002046
:10A30C00E4070020EC070020EC070020F4070020F5
:10A31C00F4070020FC070020FC07002004080020A4
:10A32C00040800200C0800200C0800201408002051
:10A33C00140800201C0800201C0800202408002001
:10A34C00240800202C0800202C08002034080020B1
:10A35C0034080020FFFFFFFF000002004300000054
:10A36C0000000000000000000000000000000000E1
:10A37C00000000000000000000000000430000008E
:10A38C0000000000000000000000000000000000C1
:10A39C00000000000000000000000000430000006E
:10A3AC0000000000000000000000000000000000A1
:10A3BC00000000000000000000000000430000004E
:10A3CC000000000000000000000000000000000081
:10A3DC00000000000000000000000000430000002E
:10A3EC000000000000000000000000000000000061
:10A3FC00000000000000000000000000430000000E
:10A40C000000000000000000000000000000000040
:10A41C0000000000000000000000000043000000ED
:10A42C000000000000000000000000000000000020
:10A43C00000000000000000000000000817F000010
:10A44C00397B000000000000AC990000A8990000C6
:10A45C00D0940000D0940000D0940000D094000060
:10A46C00D0940000D0940000D0940000D094000050
:10A47C00D0940000FFFFFFFFFFFFFFFFFFFFFFFF78
:10A48C00FFFF000001004153434949000000000058
:10A49C0000000000000000000000000000000000B0
:10A4AC000000000000004153434949000000000037
:10A4BC000000000000000000000000000000000090
:08A4CC00000000000000000088
:04000003000026B91A
:00000001FF
